:10800000000001209107010001DA000001DA000000
:1080100001DA000001DA000001DA000000000000CF
:1080200000000000000000000000000001DA000075
:1080300001DA00000000000001DA0000AD85000058
:1080400001DA000001DA000001DA000001DA0000C4
:1080500001DA000001DA000001DA000001DA0000B4
:1080600001DA000001DA000001DA000001DA0000A4
:1080700001DA000001DA000001DA000001DA000094
:1080800001DA000001DA000001DA000001DA000084
:1080900001DA000001DA000001DA000001DA000074
:1080A00001DA000079CC000001DA000001DA0000FA
:1080B00001DA000001DA000001DA000001DA000054
:1080C00001DA000001DA000001DA000001DA000044
:1080D00001DA000001DA000001DA000049C80000FE
:1080E00001DA000001DA000001DA000001DA000024
:1080F00001DA000001DA000001DA000001DA000014
:1081000001DA000001DA000001DA000001DA000003
:1081100001DA0000A9EC000001DA000001DA000039
:1081200001DA000001DA000001DA000001DA0000E3
:1081300001DA000001DA000001DA000001DA0000D3
:1081400001DA000001DA00001187000001DA000006
:1081500001DA000001DA000001DA000001DA0000B3
:1081600001DA000095C8000001DA000001DA000021
:1081700001DA000001DA000001DA000001DA000093
:0881800001DA000001DA000041
:10840000FFFFFFFFFFFFFFFFFFFFFFFF7EF9FFFF03
:1084100010B5054C237833B9044B13B10448AFF3BE
:1084200000800123237010BD0086FF1F00000000A4
:10843000440F010008B5064B1BB106480649AFF3CF
:1084400000800648036813B1054B03B1984708BD87
:1084500000000000440F01000486FF1F6885FF1F15
:108460000000000080F31188704741F238022C4B65
:10847000995841F4785199502A4A927902F00C02A5
:108480000C2A4CD041F244022749995003F5583345
:108490009A78120703D59A7842F008029A70204B16
:1084A000224941F24402995041F204015A5842F4DF
:1084B000803242F0C0025A501A6842F440221A60D8
:1084C00003F5E83324225A70194A80211170A22240
:1084D0001A70DA7802F01F02DA7003221A71002291
:1084E0005A719A799007FCD59A79D106FCD40D4B34
:1084F0009A7902F00C02082AF9D140225A719A792D
:1085000002F00C02082AFAD1064B9A795206FBD5E2
:1085100022221A709A7902F00C020C2AFAD17047C2
:1085200000700440004006400000330100001301C9
:1085300000500640184B5A7902F0E0025A711A793D
:1085400002F0F8021A71A3F55B33A3F570731A6891
:1085500042F004021A60114A136823F0784323F0B2
:10856000010313600E4B1A7802F08C0242F05002A5
:108570001A705A7802F09C0242F040025A709A78BF
:1085800002F0E6029A70074A00231370064A82F846
:10859000353383F31188704700F0074000D0004066
:1085A00000D0074000E0074000E100E0104B6846C3
:1085B0001A6820F0070101328D4601B51A600D4B93
:1085C0001A6801321A600C4B1A683AB11A68013AFB
:1085D0001A601B6813B9094B01221A70084B1A68FC
:1085E00012B11A68013A1A60BDE801408546704729
:1085F0001C86FF1FE895FF1F1C93FF1F1893FF1F8A
:108600002093FF1F024B034A5A6007221A607047EB
:1086100010E000E000770100014B1868704700BFD0
:108620001C86FF1F072888BF0020134B134A53F8EE
:10863000203010B5124CB4FBF3F441F22803422071
:10864000D15841F48061D1500E4B4FF440729A637F
:10865000DA6305F0EDF90C4B0022DA709A709A712A
:10866000DA725A71C4F30422E4B21A705C70DA78D8
:1086700042F02C02DA7010BDF80C010000700440CA
:10868000C0C62D0000B0044000A00E40094B1A687F
:1086900059680132202A08BF00228A4208D019688E
:1086A000194408721A60044BDA7842F08002DA70DA
:1086B000704700BF2086FF1F00A00E400A4B996A3A
:1086C000DA6A91420CD09A6A511C1A44996292F863
:1086D000302002709A6A202A04D100229A6201E0B6
:1086E00000207047012070472086FF1F044B1A7836
:1086F00002F0FF0012B100221A700120704700BF83
:108700001893FF1F014B1865704700BF2086FF1F9D
:10871000684620F007018D4631B527480179C9B276
:108720008C0615D5254BDA6A9C6A0132202A08BFCF
:108730000022A24206D0DD6AC4795819E4B280F85A
:108740003040DA621E4A052010601A6D1D4B1A6017
:108750004A0608D51C4B4FF480529A60164BDA78C3
:1087600002F0BF02DA700B0621D5164B1968F1B979
:10877000124B18685A68904214D0134A4FF4805034
:1087800050605A68501C1A445860107A0A4AC0B2A5
:10879000D0715868202808BF5960D37843F040034F
:1087A000D37004E0044BDA7802F07F02DA70BDE89F
:1087B00031408546704700BF00A00E402086FF1F55
:1087C0001C93FF1F2093FF1F80F00F4062B670477D
:1087D00072B6704762B6704772B670474FF0E023CA
:1087E00008B1034A00E0034AC3F80C2D704700BFEC
:1087F0000400FA050100FA0513B53F4A3F484FF45B
:10880000807306214360836091600E215161A2F55F
:1088100035224FF4002153629364D364136553658A
:10882000936502F53522403251619160344A4FF42C
:10883000907151621363936402F5342280324FF4D5
:10884000905191604FF48021516001F59051516138
:108850002C4A40F20311116051609160D1601161A6
:1088600051619161D16102F53322C032002454611B
:10887000254A2649136153619361936602F53222BA
:1088800002F580729160516103600A21C360224643
:10889000234619480824446000240194019CB4F53F
:1088A0007A7F02D2019C0134F7E70069C4071248BD
:1088B0004FF00804846048BF013200240194019CF9
:1088C000B4F57A7F02D2019C0134F7E70069C00752
:1088D00058BF01330139DCD10A2A0D4A03D10A2BD2
:1088E00001D1012300E000231370044B4FF4E06238
:1088F0001A60DA6002B010BD00F00F400090044032
:1089000000B0044000C0044000D0044070000004E7
:108910005893FF1F104B1B7882B0D3B10F4B02222C
:108920009A6004225A600022019201990C4A9142F5
:1089300002D8019A0132F7E702225A6004229A60B3
:1089400000230193019A064B9A42E7D8019B013319
:10895000F7E702B0704700BF5893FF1F00F00F40C9
:108960001FA1070003280DD8DFE800F00204060865
:10897000102205E0202203E0402201E04FF0806257
:10898000014B5A60704700BF00F10F4003280DD81B
:10899000DFE800F002040608102205E0202203E0D0
:1089A000402201E04FF08062014B9A60704700BFA7
:1089B00000F10F4038B50546002445FA04F3DB0703
:1089C000E0B202D5FFF7CEFF01E0FFF7DFFF013491
:1089D000082CF2D138BD08B5032813D8DFE800F021
:1089E00002040608002004E0012002E0022000E06A
:1089F000032003F0BDFF43F27C03984294BF0020A4
:108A0000012008BD002008BD032817D8DFE800F0CA
:108A100002070C110A4B1868C0F300107047084B8E
:108A20001868C0F340107047054B1868C0F38010F9
:108A30007047034B1868C0F3806070470020704790
:108A400000F10F4038B500242546E0B2FFF7C3FF20
:108A500018B10123A3401D43EDB20134082CF4D119
:108A6000284638BD024B1869C043C0B2704700BFEA
:108A7000C0F00F4037B50446FFF7CEFD0546FFF7BF
:108A8000CBFD401B0028B8BF40420128F7DD002085
:108A9000012C8DF804008DF8050008D005D3022CB8
:108AA0000CD1942001A9224604E0902000E09220FD
:108AB00001A9022204F0AAF99DF80400030648BFA8
:108AC00060F0FF0003B030BD08B5082003F050FF90
:108AD0005E2804D9104B1A784AB9012206E0082012
:108AE00003F046FF542802D80B4B00221A700820CE
:108AF00003F03EFFA92804D9084B4FF400725A60D6
:108B000008BD082003F034FF952803D8034B4FF429
:108B100000729A6008BD00BF7486FF1F80F00F408E
:108B2000034B1878013801288CBF002001207047C2
:108B30007486FF1F034B1878012806BF02221A70A3
:108B4000002070477486FF1FC0B204F0A7BEC0B2F9
:108B500004F092BE08B506F0ABFE05F073F905F01F
:108B600023F9BDE8084006F025BF38B5054605F0F5
:108B700071F808280AD900242819013405F0EAF808
:108B8000092CF9D105F01AF9012038BD002038BDB3
:108B9000092105F07FB8002005F008BB224A41F208
:108BA0003C030120D15841F44051D1501F4B204982
:108BB00018601A680A431A601E4ADA601A61DA6A93
:108BC00042F08052DA621A6822F001021A601A68D2
:108BD00022F000621A60184A4FF400731360536069
:108BE0009360D360136153619361D361A2F5F03256
:108BF00010601068014311601049D16001F5200137
:108C00001161D16A41F08051D162116821F00101F6
:108C10001160116821F00061116002F5E832936281
:108C2000D3621364536470470070044000C0024074
:108C3000000C1F800300013E00B004400400513EC0
:108C4000FF2800F03F031AD82C4872B141F00061B0
:108C500041EA03434363294BDA6A002A1946FADAE8
:108C6000CA6A264BD200FBD541E041F0004141EAFF
:108C700003434363214BDA6A002AFBDA37E0B0F59D
:108C8000007F1AD21E4872B141F0006141EA0343ED
:108C900043631B4BDA6A002A1946FADACA6A184B90
:108CA000D000FBD523E041F0004141EA0343436398
:108CB000134BDA6A002AFBDA19E0124872B141F06C
:108CC000006141EA034343630E4BDA6A002A194606
:108CD000FADACA6A0B4BD200FBD508E041F000413A
:108CE00041EA03434363074BDA6A002AFBDA986BD5
:108CF000DA6A42F01042C0B2DA62704700C0024045
:108D000000D0024000C00A4010B5FFF785FC0446C1
:108D1000FFF782FC001B0028B8BF40420628F7DDA1
:108D200010BD07B5030A8DF805008DF80610032263
:108D300001A9A0208DF8043004F03EF8FFF7E4FF0D
:108D400003B05DF804FB2DE9F04100238AB08846AA
:108D500016461C46B4421DD00AAA1A445D1C18F8D7
:108D6000041002F8221C2F18FA0602D0721E944238
:108D70000DD1020A8DF804208DF8050001A9DA1C36
:108D8000A02004F019F80025FFF7BEFF3846013493
:108D90002B46DFE70AB0BDE8F0811FB5030A0222C7
:108DA00003A98DF80C308DF80D0000920B46A02021
:108DB00004F056F89DF80C0005B05DF804FB1FB5F3
:108DC0000B46010A8DF80C108DF80D00009203A9D6
:108DD0000222A02004F044F805B05DF804FBC0EBCB
:108DE000C00000F5B0400722FFF7ADBFC0EBC000E8
:108DF00000F5B0400722FFF7E2BF30B500238BB08B
:108E000001AD00225A550133222BF9D14FF4B04461
:108E1000230A8DF8054029462222A02020348DF80F
:108E2000043003F0C9FFFFF76FFFB4F5803FEFD1C7
:108E30000BB030BD13B50C46C0EBC000072200F5E7
:108E4000B0406946FFF7BBFF9DF8002023789A42A7
:108E500011D19DF8012063789A420CD19DF802202F
:108E6000A3789A4207D1DDF80300D4F80330C31A7F
:108E70005842584100E0002002B010BD704713B5C1
:108E800045F2FF70FFF789FF552803D12A4B1B7865
:108E9000002B3BD045F2FF700021FFF742FFFFF7A8
:108EA000ACFF002025494022FFF74DFF402002463D
:108EB0002349FFF748FF802021494022FFF743FF65
:108EC000C0201F494022FFF73EFF002301934FF4CB
:108ED000D364204601A90422FFF735FF043440F68D
:108EE00078039C42F5D1002301934FF4FF642046A0
:108EF00001A90422FFF727FF043440F6D8039C425F
:108F0000F5D145F2FF705521FFF70BFF00200B490B
:108F10004022FFF754FF402002460A49FFF74FFF67
:108F2000802009494022FFF74AFFC020074940221C
:108F3000FFF745FF02B010BD5893FF1F0C80FF1FC5
:108F4000280D01007093FF1FB093FF1FF093FF1FC8
:108F500073B5C54EB4787278022C354600F2FC82A7
:108F6000A32A00F0048375D8132A00F0D88135D8DD
:108F7000072A00F0658115D8022A00F0108108D870
:108F8000002A00F00081012A40F0CE8320462121F2
:108F9000FEE0052A00F0378100F24781042A00F044
:108FA0001881C1E30F2A00F09B8108D80D2A00F038
:108FB000778100F285810C2A00F06281B4E3112AE6
:108FC000AA4B00F0988100F2A08153F82430D6F823
:108FD00003009847252102462046DBE01B2A00F0CB
:108FE000F18118D8172A00F0B6810ED8152A00F0A2
:108FF000CD8000F29E819D4BD6F8030053F82430BB
:1090000098472B2102462046C4E0192A00F0BD8172
:1090100040F2AB81C6E1212A00F0FC8110D81F2A62
:1090200000F0D98100F2E8811C2A40F07D83D6F857
:1090300003102046C9B202B0BDE8704004F04CB93C
:109040008C2A00F00282A22A00F088827F2A40F057
:109050006B83EEE1B82A00F01E834AD8AB2A00F0F9
:10906000E9821FD8A72A00F0CA820DD8A52A00F0ED
:10907000878200F2B082D6F803102046C9B202B04F
:10908000BDE8704004F05EB9A92A00F0C18200F288
:10909000C882D6F803102046C9B202B0BDE87040BD
:1090A00004F06EBAB12A00F0E08210D8AD2A00F0C8
:1090B000D382C0F0C882AE2A40F03683D6F80310BF
:1090C0002046C9B202B0BDE8704004F049BAB52AE2
:1090D00000F0C581B62A00F03A82B32A40F024831A
:1090E000D6F803102046C9B202B0BDE8704004F0C3
:1090F00065B9C92A00F0D58121D8BC2A00F00283C5
:109100000DD8BA2A00F0D08200F2E682D6F8031019
:109110002046C9B202B0BDE8704004F095B8C22A3A
:1091200000F0AA81C32A00F0B181C12A40F0FC827C
:109130004F4B03EB8414D6F803302372F7E2D22AA4
:1091400000F0C5810FD8CC2A00F0E582D12A00F0CA
:10915000B681CA2A40F0E882454BD6F8032003EBDB
:1091600084135A83B9E1D62A00F0BD81FF2A00F0AA
:10917000CB81D42A40F0D8823D4B03EB8414D6F83F
:1091800003302362D3E220462D2101E020462C212A
:10919000D5F8032002B0BDE8704003F07DBFD6F8DB
:1091A0000330002BC8BF01222046202103F074FFAA
:1091B000B478304BD6F8030001221A552B4B002807
:1091C000B8BF404253F82430984727210246204632
:1091D000E0E7264ED5F8030056F824300028B8BF43
:1091E0004042984706EB84042021E060A87803F011
:1091F00083FF002840F09B821B4B987806EB80068B
:109200002721F268C6E71C4BD6F8030000221A5546
:10921000164B03EB84039B699847184B43F82400D3
:10922000B078262153F82020B4E72046102103F01F
:1092300063FFF2780346D208B0780092DAB20AE00F
:109240002046102103F058FF0346C3F30722B078ED
:109250000092F278D208019210210022C3F3074352
:1092600003F0DEFE63E200BFD094FF1F7886FF1F8D
:109270007093FF1F4693FF1FCC94FF1FC094FF1FE6
:109280003421204603F038FFD6F80330024634215B
:10929000B07813B942F002027CE722F0020279E7CB
:1092A0003421204603F028FFD6F80330024634214B
:1092B000B07813B942F001026CE722F0010269E7CD
:1092C0003421204603F018FFD6F80330024634213B
:1092D000B07813B142F010025CE722F0100259E7B7
:1092E000B14BD6F8030003EB84039B699847242114
:1092F000024620464EE703EB8403D6F803009B6941
:10930000984728210246204644E703EB8403D6F819
:1093100003009B6998472A21024620463AE7A24B60
:10932000D6F8030053F824309847232102462046FC
:1093300030E7D6F80330002BC0F20E819B4A02EBD7
:109340008414227E012A03D0184604F021FB034630
:10935000A8781521B9E1944BD6F8030053F82430CE
:10936000984733210246204614E73421204603F073
:10937000C3FED6F8033002463421B07813B142F070
:10938000080207E722F0080204E73421204603F030
:10939000B3FED6F8033002463421B078002B00F03B
:1093A000AE81A9E13421204603F0A6FED6F80330B1
:1093B00002463421B07813B142F40062EAE622F4A6
:1093C0000062E7E6D6F803102046C9B202B0BDE855
:1093D000704003F06FBF1021204603F08DFEB2787D
:1093E000F378C0F30721C0B200910190102110461C
:1093F00003F00F03002233E76E21204603F07CFECA
:109400003179B27801F003010091F1780191C0F354
:1094100007430AE06E21204603F06EFEC0F30721E9
:10942000C0B2B278F3780091019010466E2100220C
:1094300016E7D6F80330022B00F28E805A4B1C44FC
:109440005B4BDB7884F8243071E1D6F80310C1F16E
:1094500008012046C9B203F009FFB0783EE0D6F813
:109460000300002878DB504B53F8243098474F4BCB
:1094700003EB841420615AE14B4BD6F8030053F8F8
:1094800024309847A401494B185150E1464BD6F877
:10949000030053F824309847444B03EB8414606076
:1094A00045E13821204603F027FED6F8033000F4CA
:1094B000806223F48063B07838211A436AE6D6F8D4
:1094C0000310204602B0BDE8704003F0A4BD374B46
:1094D000D6F8032003EB8413DA61204602B0BDE81E
:1094E000704003F0FDBCD6F8030006F0CBFB2CA3C4
:1094F000D3E9002306F056FD07F06EFB06F0C2FE2E
:1095000011210246204645E6D6F803308BB1012BE7
:1095100022D1264A02EB84121376234B254A43F8C4
:10952000242003EB8404244BA362244BA361244B2B
:109530000BE01E4A02EB841213761B4A214B42F8C1
:10954000243002EB8404A362A3616363EFE0D6F8E6
:109550000330002B80F292800422E6E0D6F803105C
:109560002046C9B202B0BDE8704003F05BBED6F839
:1095700003102046C9B202B0BDE8704003F0BEBE81
:10958000204603F077FFD6F80310E8B9B078C9B2E7
:1095900002B0BDE8704003F033BE00BFAFF30080FF
:1095A0002D431CEBE236FA3F7886FF1F7093FF1FB6
:1095B000D094FF1F2DD9000091D9000069D9000077
:1095C000D1D90000F9D90000B078C9B202B0BDE825
:1095D000704003F0C9BE204603F04CFFD6F80310DC
:1095E00030B9B078C9B202B0BDE8704003F0F6BD42
:1095F000B078C9B202B0BDE8704003F0CDBED6F875
:1096000003102046C9B202B0BDE8704003F0CCBDE3
:10961000D6F803102046C9B202B0BDE8704003F08E
:109620006ABFD6F803102046C9B202B0BDE8704048
:1096300003F073BFD6F803102046C9B202B0BDE8EC
:10964000704003F046BFD6F803102046C9B202B0FE
:10965000BDE8704003F073BFD6F803102046C9B2CE
:1096600002B0BDE8704003F09DBFD6F8031020465D
:10967000C9B202B0BDE8704003F00ABE2D4A02EB49
:109680008414227E012A03D0184604F081F903468F
:10969000A878142119E0D6F803102046C9B202B008
:1096A000BDE8704003F03CBED6F80330002BFFF657
:1096B00053AF204A02EB8414227E012A03D01846BD
:1096C00004F066F90346A8781321002BCABF1A4A92
:1096D0001A4A92FBF3F25DE5D6F803102046C9B2B0
:1096E00003F0EFFF0021B07803F006FDD6F8031079
:1096F0000246B07819B1002142F004024AE522F096
:10970000040247E5D6F803102046C9B202B0BDE80E
:10971000704003F0E6BFD6F803102046C9B202B08D
:10972000BDE8704003F085BF0322054B1A7002B0FC
:1097300070BD00BF7093FF1F0024F400B50010003F
:10974000EC95FF1F38B59D4A90780228144600F02A
:10975000F480032800F0F880002840F09C815378C2
:109760004D2B00F0998032D8452B71D015D8412B64
:1097700062D006D8402B40F08C8145F2FF70D17842
:109780005DE0422B5FD0442B40F083818C49D2F8BE
:10979000033041F81C3F1C2065E0492B65D00CD8F4
:1097A000462B5AD0472B40F07481854DD2F80330B8
:1097B0002946082041F8083F90E04B2B61D04C2B04
:1097C00040F067817E4BD1789970022037E0542BAE
:1097D00000F08E8019D8512B6AD009D84F2B60D059
:1097E000502B40F05681764BD1789975162026E0A3
:1097F000522B6CD0532B40F04C81714DD2F803307A
:109800002946102041F8103F68E0842B00F08B803F
:1098100009D8552B77D0832B40F03B81694BD2F888
:1098200003201A6438BD852B00F08280FF2B40F0A6
:109830003081D278644B30E1614BD1781970BDE84A
:109840003840FFF76EBA5E4BD17859700120F6E7C9
:109850005B4BD17859710520F1E75949D2F80330B3
:1098600041F80C3F0C20042259E0D278544B0AB93D
:10987000DA7503E055490122DA754A601720D97D6F
:10988000DDE74F4CD178E1700320FFF74AFAE0782A
:10989000BDE83840FEF736BF494BD17859751520E1
:1098A000CDE7D2F80310464BC9B259761920C6E766
:1098B000434B1A7D12F0010F1D4604D0E378DB07FD
:1098C00001D4FFF79AFAE17829751420B7E73C49EB
:1098D000D2F8033041F8203F2020C4E70422FFF7EC
:1098E00032FA687929892A8ABDE8384003F070B8CD
:1098F000D2F80330012B00F2CE803149D37801F841
:109900001A3F1A200AE0D2F80330012B00F2C3807C
:109910002A4B2B49DB7801F81B3F1B200122BDE8B5
:109920003840FFF710BA2A4BD2F803201A6038BD2E
:10993000244BD2F803205A6438BD5178254BD2F815
:10994000032043F8212038BD53782E2B00F2A1804C
:10995000DFE803F018212A9F9F9F9F9F9F44494E55
:109960009F9F9F9F9F9F9F9F9F9F9F9F9F9F9F5353
:10997000595F656B719F9F9F9F9F9F777C81868BAF
:1099800090959A00144BD4F803201A60FEF744FE19
:109990000C4B986438BD104BD4F803205A60FEF786
:1099A0003BFE084BD86438BD0B4BD4F803209A60BB
:1099B000FEF732FE034B186538BD00BFD094FF1F81
:1099C0000C80FF1F7886FF1FE695FF1FEC95FF1F99
:1099D000E895FF1FF895FF1F4094FF1F304BD4F808
:1099E0000320DA6038BD2E4BD4F803201A6138BD4D
:1099F0002B4BD4F803205A6138BDD4F80320284BF0
:109A0000D2B21A7638BDD4F80320254BD2B2DA761A
:109A100038BDD4F80320224BD2B25A7638BDD4F8E0
:109A200003201F4BD2B21A7738BDD4F803201C4B49
:109A3000D2B29A7638BDD4F80320194BD2B25A77F5
:109A400038BD174BD4F803201A6238BD144BD4F834
:109A500003205A6238BD124BD4F803209A6238BDF5
:109A60000F4BD4F80320DA6238BD0D4BD4F8032035
:109A70001A6338BD0A4BD4F803205A6338BD084B2B
:109A8000D4F803209A6338BD054BD4F80320DA6379
:109A900038BD032200E00422024B1A7038BD00BF1B
:109AA0004094FF1FEC95FF1F2DE9FF41C14EC24FAF
:109AB00032787A7064233B70212AD6F803307B60B9
:109AC00035463C4601F073825AD80E2A00F0BB8618
:109AD0002AD8072A00F02D8511D8032A00F03581F5
:109AE00007D8012A00F0BE80022A00F0F28001F0BF
:109AF0003CBD052A00F0538240F2458153E20A2A18
:109B000000F01F8509D8082A00F01385092A41F0C2
:109B10002C85FFF717FE01F02ABD0C2A00F04E86B7
:109B200040F2358600F060BE182A01F00B8012D892
:109B3000142A00F0508707D80F2A00F0A386132AB2
:109B400000F0108701F011BD162A00F0E98740F2FD
:109B5000648700F0E9BF1C2A01F0208106D81A2A88
:109B600001F00E8040F2FB8701F01BB81F2A01F0C4
:109B7000688101F2C1811E2A01F0158101F0F5BC56
:109B8000802A01F0F18238D8402A01F0DB821BD80C
:109B9000242A01F067820DD8222A01F05C82232A50
:109BA00041F0E384854B1B68C6F80330FFF7CAFD1C
:109BB00001F0DDBC262A01F08C82C1F08082272AC8
:109BC00001F0AE8201F0D1BC442A01F0C48208D871
:109BD000422A01F0BA8201F2BB8202F0A4F901F03C
:109BE000C6BC462A01F0BD82C1F0B882472A41F0C6
:109BF000BC8402F0AAF901F0BABC872A01F086837E
:109C000017D8832A01F0DC820BD8812A01F0C282A6
:109C1000822A41F0AA846A4B022283F8542001F080
:109C2000A6BC852A01F0FD82664A41F2E98201F074
:109C3000FDBA8C2A01F0C18309D8892A01F08F83EB
:109C4000C1F02F838A2A01F0A18301F08EBCF22A91
:109C500001F03D84FF2A01F07F848D2A41F0858444
:109C600001F0CFBBB078022836D8574B574E0024AE
:109C70001C54574B1C54335C3BB1564B262153F8B4
:109C8000202003F009FAAB78F454AC78524BD5F8A5
:109C9000030001261E554A4B0028B8BF404253F826
:109CA0002430984727210246204603F0F5F9D5F8DD
:109CB0000330A878002B4FF00002DCBF0223019391
:109CC0000092C8BF01962021134603F0A9F901F0C4
:109CD0004EBCB078022803D90423237001F047BC9E
:109CE000394B3A4E00241C54394B1C54335C43B15D
:109CF000384B262153F8202003F0CEF92D4B9B78CA
:109D0000F454AC78344BD5F8030001261E552C4B87
:109D10000028B8BF404253F8243098472721024614
:109D2000204603F0B9F9D5F80330A878002B4FF09E
:109D30000002C4BF022301930092D8BF01962021E4
:109D4000134603F06DF901F012BCB0780228C3D8B5
:109D500002F06CFDB078204B01221A54272100221A
:109D600003F09AF900240223B07801932246234697
:109D70000094202103F054F9B378134AD454144AC0
:109D8000D45401F0F4BBB078022804D9094A5278BF
:109D9000022A41F0EC830C4A064F002616540C4A66
:109DA00016546A78012A43D018D3022A00F0828020
:109DB000F1E000BFD094FF1FEC95FF1FD895FF1F67
:109DC0007886FF1F0C80FF1F4393FF1FCC94FF1F5B
:109DD0006893FF1FC094FF1F4693FF1FB54C235C81
:109DE00043B1B54B03EB80032721DA6803F054F944
:109DF000BB78E654A878B14C235C4BB1B04B26211C
:109E000053F8202003F048F9AE4B9B780022E2542F
:109E1000A878D5F803202D2103F03EF90022A87878
:109E2000009201922021134603F0FAF801F09FBB43
:109E3000A14A1318904693F82430012B07D004D37D
:109E4000022B08D103F0E4F804E02D2100E02121E9
:109E500003F052F90646A878964F3B5C4BB108EBED
:109E600080032721DA6803F017F9964B9B780022CC
:109E7000FA54A878914F3B5C4BB1914B262153F893
:109E8000202003F009F98F4B9B780022FA54D5F873
:109E90000330A8781E442D21324603F0FDF800223D
:109EA000A878009201922021134603F0B9F8666069
:109EB00001F05DBB142B6ADC030636D53446AB7863
:109EC0002341DF072CD57B4FE35DE6B243B17E4BE8
:109ED000304653F82420272103F0DEF80023E35511
:109EE000764FE35D43B1764B304653F8242026216C
:109EF00003F0D2F80023E355D5F80330734A03EB9F
:109F000043032344304652F823202D2103F0C4F8A4
:109F100000220092019230462021134603F080F87F
:109F20000134032CCBD101F022BB02282FD8614C85
:109F3000235C43B1604B03EB80032721DA6803F015
:109F4000ABF8BB78E654A8785C4C235C4BB15C4B17
:109F5000262153F8202003F09FF85A4B9B780022CB
:109F6000E254D5F80330A878584A03EB430303447E
:109F70002D2152F8232003F08FF80022A8780092B8
:109F800001922021134603F04BF801F0F0BA0423AC
:109F9000237001F0ECBA0323237001F0E8BAFEF756
:109FA000D7FF01F0E4BAB078737802283FF694AE98
:109FB000A42B00F0478200F2A080122B00F09881C1
:109FC00041D8082B00F065811AD8032B00F042819C
:109FD00006D8012B00F0338100F236812D212FE1CC
:109FE000052B00F04681C0F03E81062B00F04A812F
:109FF000072B40F08682102103F07EF8C0B246E1C4
:10A000000D2B00F05B810DD80A2B00F04B81C0F0C6
:10A0100046810B2B00F048810C2B08BF342100F047
:10A0200045816EE20F2B00F05781C0F04F81102B5D
:10A0300000F05881112B40F064821F4B03EB80032A
:10A0400028215D6B0BE11C2B00F07E811FD8172BA4
:10A0500000F062810DD8142B00F05681C0F04E81C3
:10A06000152B00F05781162B08BF152100F0218217
:10A0700047E2192B00F05C81C0F054811A2B00F0EC
:10A080005D811B2B40F03D8203F0E6F9DAE0212BE5
:10A0900000F06A811CD81E2B00F06081C0F057814F
:10A0A0001F2B00F05B81202B08BF6E2100F08C81FC
:10A0B00027E200BF4693FF1F7886FF1FCC94FF1F47
:10A0C000C094FF1FD094FF1F8486FF1FDC94FF1FE6
:10A0D0008C2B00F04E8107D87F2B40F01282BD4BB5
:10A0E000184490F824300AE2A22B00F0A881A32B98
:10A0F00040F0078203F0BEF9A4E0BB2B00F0EF8133
:10A1000048D8AD2B00F0C68117D8A82B00F0B68137
:10A1100005D8A62B00F0A48140F29781ABE1AA2BD1
:10A1200000F0B281C0F0AD81AB2B00F0B081AC2B60
:10A1300040F0E78103F05DFA84E0B52B00F01E816A
:10A1400015D8B12B00F0A98105D8AE2B40F0D981EC
:10A1500003F056FA76E0B32B00F0A281B42B40F066
:10A16000D0816F2102F0C8FFC0F304406AE0B82B31
:10A1700000F0998105D8B62B08BF142100F0998111
:10A18000BFE1B92B00F09281BA2B08BF132100F078
:10A190009081B6E1CA2B00F0118120D8C22B00F0CB
:10A1A000F6800FD8BD2B00F0A081C0F09B81BE2BA4
:10A1B00000F09D81C12B40F0A481874B03EB801000
:10A1C000037A9CE1C42B00F0F380C0F0E880C52B3B
:10A1D00000F0F080C92B08BF382131D091E1D12B9C
:10A1E00000F0168114D8CE2B00F0ED8005D8CC2BD2
:10A1F00040F0878103F084FA24E0CF2B00F0F48054
:10A20000D02B40F07E816F2102F076FF000E19E026
:10A21000D42B00F0008107D8D22B40F072816E4B16
:10A2200003EB8010C3696AE1D62B00F0F980FF2BA5
:10A2300040F06781684B03EB8010037E5FE12121D2
:10A2400002F05AFF60605EE1624B03EB800327215E
:10A250009D6A04E05F4B03EB800322219D6A02F0BC
:10A260004BFFA847EEE75B4B03EB8000836AC068B7
:10A2700006E0584B594A03EB800352F820005B6B11
:10A280009847DFE7102102F037FFC0F30720C00036
:10A29000D8E7352102F030FFC0F34020D2E703F0C9
:10A2A0002DFBCFE7352101E0352108E002F024FF46
:10A2B00010F0020F14BF0023012320E1342102F02B
:10A2C0001BFF00F0010080F00100BBE7342102F029
:10A2D00013FFC0F30010B5E73E4B03EB80032421CE
:10A2E0005D6BBCE73B4B03EB800325219D6AB6E722
:10A2F000384B03EB80032A215D6BB0E7354B03EB52
:10A30000800323219D6AAAE7324B03EB80032B21B4
:10A310009D6AA4E72C2193E72E4B03EB80033321A6
:10A320009D6A9CE7342102F0E7FEC0F3C00089E794
:10A33000342102F0E1FEC0F3800083E7342102F013
:10A34000DBFEC0F3C0207DE703F08DF87AE7214BF8
:10A3500003EB80039D6A01F007FE82E7102102F003
:10A36000CBFEC0F303406DE76E2102F0C5FE001482
:10A3700068E703F063F8C0F1080063E7154B164A7D
:10A3800003EB800302EB80109B6A006978E7114BB6
:10A39000114A03EB800380019B6A105870E70D4B54
:10A3A0000D4A03EB800302EB80109B6A406867E76D
:10A3B0000B4B00E00B4B53F82030A0E0064B03EBB7
:10A3C0008010438B9BE06F2102F096FEC0F30900E2
:10A3D00038E700BF7886FF1F7093FF1FC094FF1FF0
:10A3E0002C93FF1F3494FF1FB378A54AD05C002143
:10A3F000796010B1A34801254560D154A24AD15CCF
:10A4000019B1616841F0020161600021D1547AE024
:10A4100002F0FEFD16E79D4B03EB8010036A6EE031
:10A42000112102F069FE05F02DFC93A3D3E900236E
:10A4300005F08EFC06F040FB05F024FF02E702F079
:10A44000EFFFFFE603F024F8FCE603F013F818B979
:10A45000B07802F0DEFFF5E6B07803F020F8F1E620
:10A4600003F008F818B9B07802F0CCFFEAE6B0784B
:10A4700003F021F8E6E602F0B3FFE3E603F0CBF8E1
:10A48000E0E603F0A8F8DDE603F0ACF8DAE603F066
:10A490009BF8D7E603F0C6F8D4E602F0D6FFD1E683
:10A4A00003F010F8CEE602F0ECFFCBE602F0BFFFBF
:10A4B000C8E602F021FE002804DD754B93FBF0F0A6
:10A4C000606002E06FF07F436360AA786F4B03EB3C
:10A4D00082131B7EBBB9606803F028FAB2E603F072
:10A4E0002BF9AFE603F02FF9ACE67121A8E60021C5
:10A4F00002F002FE10F004003FF4A4AE01236360FA
:10A5000001E003232370634B1B78002B01F02F80A5
:10A51000614B62681A60614B2AB91A6842F00802FE
:10A520001A6001F024B81A6822F008021A6001F0DB
:10A530001EB8B378022B3FF6CFAB0323237001F094
:10A5400016B8B378022B00F0C580032B00F0C7804B
:10A55000002B40F004817378502B70D029D8462B03
:10A560005FD012D8422B55D007D8402B4CD0412B6E
:10A5700040F0F3804A4B1B784EE0442B4ED0452BE5
:10A5800040F0EB80464B5B7946E04B2B4ED007D832
:10A59000472B49D0492B40F0E080414BDB7D95E0D3
:10A5A0004D2B49D045D34F2B40F0D7803C4B5B7EA1
:10A5B00032E0802B52D013D8532B46D006D8512BE3
:10A5C00040D0522B40F0C980354BB5E0552B42D0DE
:10A5D0003ED3562B40F0C180314B93F824301BE022
:10A5E000832B63D007D8812B3CD0822B40F0B580E1
:10A5F0002C4B9B6D10E0852B5DD05AD3FF2B40F088
:10A60000AC80294B1B7861E045F2FF70FEF7C5FB7B
:10A610007860A6E0224B5B786360A2E0204BDB69A8
:10A62000FAE71F4BDB68F7E71D4B83E01C4BDB7839
:10A63000F2E71B4B9B78EFE7194B5B7DECE7184B80
:10A640009B7DE9E7164B1B7DE6E7154B1B69E3E7AE
:10A65000134B9B7EE0E7124BDB7EDDE7114B93F85B
:10A660005430D9E70F4B93F854301E1F7342734197
:10A67000D2E700BFAFF300802D431CEBE236FA3F78
:10A680006893FF1FEC95FF1F4393FF1F7093FF1FFD
:10A690000024F400E795FF1FD895FF1FD894FF1FF3
:10A6A0000C80FF1F7886FF1FE695FF1FA04B1B6CD9
:10A6B000B2E7A04B3BE09E4A9F49536C4B4303F5E6
:10A6C00040533933536423F00043A5E7003318BFE8
:10A6D0000123A1E77278994B53F822309CE77378F5
:10A6E000282B2BD010D8022B23D005D8F3B1012B67
:10A6F00033D1934B5B688FE7092B2ED30B2B30D9CB
:10A70000272B2AD18E4B17E02B2B1DD006D8292BB7
:10A7100017D02A2B21D18A4BDB6A7DE72D2B19D04C
:10A7200015D32E2B19D1864BDB6B75E7844B1B6839
:10A7300072E7834B9B686FE71B6A6DE7804B5B6A30
:10A740006AE77F4B9B6A67E77D4B1B6B64E77C4B3B
:10A750005B6B61E77A4B9B6B5EE7032300E00423AE
:10A760002370784B1B78002B00F00187764B6268D2
:10A770001A60764B2AB91A6842F008021A6000F093
:10A78000F6BE1A6822F008021A6000F0F0BEB37834
:10A79000022B0FD16E4B5B78372B3FF6CEAE67495D
:10A7A00003F5FF70800001EB83010422FEF7CBFA72
:10A7B00000F0DDBE04233B7000F0D9BEB378022B5D
:10A7C0000ED17378372B3FF6B8AE5C4903F5FF70B6
:10A7D000800001EB83010422FEF7F1FA00F0C7BE0E
:10A7E00004233B7000F0C3BEB07802283FF674AA81
:10A7F000574B5B78012B07D002D3022B08D01EE009
:10A8000002F00CF800F0B3BE02F010F800F0AFBE9A
:10A8100002F014F84B4B78601B78002B00F0A786F1
:10A82000494B1860494B1A6820B942F008021A6077
:10A8300000F09DBE22F008021A6000F098BE0323CB
:10A840003B7000F094BEB278022A17D170780728C6
:10A8500008D81BB9FEF79AF800F089BEFEF782F817
:10A8600000F085BEFF2840F082865D1C0ABF364B93
:10A87000D8B21878FEF79EF800F079BE04233B703A
:10A8800000F075BEB378012B1CD02BB1022B3CD14C
:10A890007078FEF7B9F813E07078082802D8FEF750
:10A8A0009AF80DE00A2807D12A4B1B6983F400733C
:10A8B000C3F340237B602AE0FF2828D1FEF7C2F8CB
:10A8C000606024E07078092802D002F051F8F7E7C0
:10A8D0000020FEF7CFF806460120FEF7CBF805462C
:10A8E0000220FEF7C7F88542D4BF0022012296421B
:10A8F00001DD2A1C00E0021C18BF01221AB9A8427F
:10A90000ACBF06462E46666001E004233B700D4B4B
:10A910001B78002B00F02B860B4B62681A600B4BE8
:10A92000D2B91A6842F008021A6000F020BE00BFD7
:10A930007886FF1FE895FF1F6D4EC641F895FF1FF3
:10A940004094FF1FE795FF1FD895FF1FD894FF1F66
:10A95000D094FF1F80F00F401A6822F008021A609E
:10A9600000F005BE7178964A092925D8DFE801F084
:10A9700005080B0E12181B1E212311680B441AE048
:10A980001168CB1A17E011684B4314E0116891FB72
:10A99000F3F310E0116891FBF3F003FB10130AE0EE
:10A9A00011680B4007E011680B4304E011684B404D
:10A9B00001E01368DB4313601268824B2AB91A68FE
:10A9C00042F008021A6000F0D2BD1A6822F00802B4
:10A9D0001A6000F0CCBD7A4A12689A42794B196825
:10A9E00004DD21F0030141F0040108E00BBF21F078
:10A9F000060121F0050141F0010141F00201196059
:10AA00002AB91A6842F008021A6000F0B0BD1A684C
:10AA100022F008021A6000F0AABD72780C2A00F237
:10AA2000A685DFE802F0071019222B343E47505963
:10AA3000626B7400634A1268140740F19885624A99
:10AA4000936500F094BD5F4A1268100700F18F858E
:10AA50005D4A936500F08BBD5A4A1268D10740F1F8
:10AA60008685594A936500F082BD564A1268D2071E
:10AA700000F17D85544A936500F079BD514A126812
:10AA8000570740F17485504A936500F070BD4D4AF8
:10AA9000126812F0050F00F06A854B4A936500F0CA
:10AAA00066BD484A1268960740F16185464A93653B
:10AAB00000F05DBD434A1268950700F05885424A90
:10AAC000936500F054BD3F4A1268D40640F14F85AB
:10AAD0003D4A936500F04BBD3A4A1268900640F13A
:10AAE0004685394A936500F042BD364A12685106E0
:10AAF00040F13D85344A936500F039BD314A126812
:10AB0000120640F13485304A936500F030BD2D4A7D
:10AB10001268D70540F12B852B4A936500F027BDBD
:10AB2000294A936500F023BD274AD16D072900F219
:10AB30001E85481C02EB8101D065906D0866936507
:10AB400000F015BD204BDA6D002A00F01085013AA7
:10AB5000DA6503EB8202126E9A6500F008BD737825
:10AB60002E2B04D8194A0121D15400F000BDFF2B2F
:10AB70007FF4E3AC144B012283F8802000F0F7BC93
:10AB800073782E2B04D8114A0021D15400F0EFBC69
:10AB9000FF2B7FF4D2AC0C4B002283F8802000F016
:10ABA000E6BC094C94F88120E2B95E1C4FF00A0221
:10ABB0000ED1034B1B685A43C4F884200BE000BF3E
:10ABC000D895FF1FD894FF1F7886FF1F9194FF1F11
:10ABD0005343C4F88430FDF71FFD0123C4F88800F7
:10ABE00084F881306B78042B00F2C184DFE803F035
:10ABF000034878A81B00FDF70FFDD4F88820D4F88F
:10AC00008410B64B801A80EAE072A2EBE0728A42AE
:10AC100004D9002283F8812000F0A9BC9A6D013A82
:10AC20009A6500F0A4BCA87801F008FE40B9AC4BCE
:10AC300084F881001A6822F010021A6000F097BCB4
:10AC4000D4F88430A54DB3B1FDF7E6FCD5F88830D3
:10AC5000D5F88420C01A80EAE073A3EBE073934236
:10AC600009D9002385F881309D4B1A6842F0100203
:10AC70001A6000F07CBCA36D013BA36500F077BCBB
:10AC8000A878352102F038FA10F4007609D00023B4
:10AC900084F88130924B1A6822F010021A6000F09A
:10ACA00066BCD4F884308D4DABB1FDF7B5FCD5F85A
:10ACB0008830D5F88420C01A80EAE073A3EBE073F3
:10ACC000934208D9864B85F881601A6842F01002D9
:10ACD0001A6000F04CBCA36D013BA36500F047BCBB
:10ACE000A878352102F008FA10F0010609D00023F7
:10ACF00084F881307A4B1A6822F010021A6000F052
:10AD000036BCD4F88430754DABB1FDF785FCD5F871
:10AD10008830D5F88420C01A80EAE073A3EBE07392
:10AD2000934208D96E4B85F881601A6842F0100290
:10AD30001A6000F01CBCA36D013BA36500F017BCBA
:10AD4000A878352102F0D8F910F0020609D00023C6
:10AD500084F88130624B1A6822F010021A6000F009
:10AD600006BCD4F884305D4DA3B1FDF755FCD5F891
:10AD70008830D5F88420C01A80EAE073A3EBE07332
:10AD8000934207D9564B85F881601A6842F0100249
:10AD90001A60ECE3A36D013BA365E8E34F4B00228F
:10ADA00083F85420E3E37678142E3FF6C6AB4D4A81
:10ADB0009778022F1AD806EB46014B4C394444F8D9
:10ADC00021304A4B9B7E002B00F0D183002E00F0F7
:10ADD000CE83013E0C207043042200F5D36002FBB9
:10ADE000070004EB8101FDF7AEFFC0E3FF2F7EF407
:10ADF00073AF3D4F86B90C25002405F28C6079199C
:10AE00002044214404220434FDF79DFF0C2CF4D18E
:10AE10000C35FC2DF0D1AAE300246B780C205A1ECF
:10AE2000504303EB4303E11800F5D36000EB8400CB
:10AE300007EB810104220134FDF785FF032CECD1DF
:10AE400095E37378142B3FF678ABB278022A19D8C1
:10AE500003EB43031A44264B23491B7851F8222065
:10AE60007A60002B00F08383224B1A601C4B22B9BE
:10AE70001A6842F008021A6079E31A6822F00802A0
:10AE80001A6074E3FF2A7EF427AF174E83B90C25AE
:10AE9000002405F28C6071192044214404220434FA
:10AEA000FDF78DFF0C2CF4D10C35FC2DF0D15EE3B9
:10AEB00000246B780C205A1E504303EB4303E11827
:10AEC00000F5D36000EB840006EB8101042201341D
:10AED000FDF775FF032CECD149E300BF7886FF1F17
:10AEE000D894FF1FD094FF1FDC94FF1F0C80FF1F1E
:10AEF000E795FF1FD895FF1F96F801809D4FB8F189
:10AF0000140F3FF61AABBE78300629D50024AB7873
:10AF10002341D9070BD5974B5E78E0B2212102F08F
:10AF2000EBF806EB46062644934B43F82600934B7A
:10AF30009B7E8BB16B787BB15A1E0C20504303EB88
:10AF400043038D4A00F5D360E11802EB810100EB69
:10AF500084000422FDF7F7FE0134032CD7D106E369
:10AF6000022E3EF6B9AE3046212102F0C5F8834BE1
:10AF7000814C9B7E08EB4808464444F82600002B91
:10AF800000F0F5827B78002B00F0F182BD78591E2D
:10AF90000C20484303EB43030422E91800F5D36077
:10AFA00002FB050004EB8101FDF7CDFEDFE27278C4
:10AFB000734B0A2A42D8DFE802F0060B11161C2454
:10AFC000292E33383C006F491A6809680A4403E0A7
:10AFD0006C491A680968521A1A602FE069491A68A0
:10AFE00009684A43F8E767491A68096892FBF1F271
:10AFF000F2E7644A1968126891FBF2F002FB101242
:10B00000EAE7604A11681A680A40E5E75D4A116894
:10B010001A680A43E0E75B4A11681A684A40DBE7AE
:10B02000584A1168C943116008E056491A680A6015
:10B0300004E0544A18681168196010601A68524B8D
:10B0400022B91A6842F008021A6090E21A6822F0E7
:10B0500008021A608BE24A4B1B68C6F80330FDF702
:10B0600077FF84E27378052B00F28182DFE803F03A
:10B0700003090F151B21444B1A6802F00F021A60D6
:10B0800075E2414B1A6822F010021A606FE23E4BE3
:10B090001A6822F020021A6069E23B4B1A6822F01B
:10B0A00040021A6063E2384B1A6822F080021A608C
:10B0B0005DE2354B1A6822F480721A6057E27278AA
:10B0C0002E2A3FF63AAA314901EB8202C2F88C30AF
:10B0D0004DE22E4B2A49D3F848210A602949D3F87A
:10B0E0004C210A60D3F8502127499A65D3F854219E
:10B0F0000A60D3F8582183F88120D3F85C21C3F883
:10B100008820D3F86021C3F88420214993F8642172
:10B11000885C08B101208854002283F8682126E267
:10B12000B278022A3EF6D8AD124B5B78142B3FF66C
:10B1300004AA03EB43031A44114B0F491B6841F85F
:10B14000223014E200F0EEFE11E200F0F9FE0EE211
:10B1500000F0F7FE0BE200F0F5FE08E200F0F3FE6F
:10B1600005E200F0F1FE02E2084B002283F85420D1
:10B17000FDE100BFD094FF1FDC94FF1F0C80FF1F78
:10B18000D895FF1FF495FF1FD894FF1F7886FF1FE7
:10B190009194FF1F727812B1012A05D00DE0A74BE0
:10B1A000012283F85420E2E1B3F5C05FBEF494AD10
:10B1B000A24981F854208B65D9E103233B70D6E185
:10B1C0009E4B002183F8801083F868119B4A02F19E
:10B1D0008C034FF0FF3043F821009948002343547B
:10B1E00001312F29F2D182F854309365D36582F86A
:10B1F0008130944A1360944A1360944A1360B6E114
:10B20000127D92070AD4B3F5C05FBEF465AD8B4AD8
:10B21000042182F85410C2F86C31A8E108233B7075
:10B22000A5E1864B002283F85420A0E18849894C8F
:10B23000927822700125B3F5C05F0D7027D2864A3F
:10B24000127D12EA050622D1184602A9FDF7CEFDAD
:10B250009DF8083063709DF80930A3709DF80A309E
:10B26000E3709DF80E3023719DF80D3063719DF8E9
:10B270000C30A3719DF80B30E37126722B46E15C14
:10B28000227A01330A44082B2272F8D16FE101239C
:10B290000021E1540133082B6E4AF9D1137813725F
:10B2A00065E17378012B1DD00AD3022B2BD1684B9B
:10B2B00001221A70684B674A9B781370002319E0CB
:10B2C000634B01221A70644B624A9B781370634B84
:10B2D000186800230133C118082B11F8011CD15440
:10B2E000F8D144E10C22FA717B718C220523BA71EA
:10B2F0003B713CE15A4901331944082B11F8091CF0
:10B30000D154F7D133E103233B7030E17378032B41
:10B3100000F22D81DFE803F0020F1B1F474B93F86B
:10B320005420FA7193F88120D3F86C31BA711A0A5B
:10B330007A713B711BE1414B93F85420FA7193F8F9
:10B3400081209B6DBA711A0A7A713B710FE13D4BF6
:10B350001B687B600BE13C4B1B687B6007E17278EC
:10B36000002A40F00481B178002940F0008140F2C9
:10B37000D242934240F0FB8045F2FF70FDF7D1FCD2
:10B38000FDF73BFD0120FDF729FAF0E07278354B1F
:10B3900002B101221A70344BEA781A70274B93F8E5
:10B3A0007011324B1970324900230B7031490B7008
:10B3B000314B19780A431A70D9E0757815B1012D0F
:10B3C0000FD01BE0042245F2FB7002A9FDF7F7FC49
:10B3D000029BD6F803209A4206BF01237B607D6062
:10B3E000C5E0B3782A2B06D145F2FB70234904222D
:10B3F000FDF7A9FCBBE003233B70B8E003233B70DF
:10B40000B5E07278032A5FD8DFE802F00802505BEB
:10B410000A480022D0F87411054632E0074AD2F8F3
:10B420007411092907D8481CC2F8740102EB810283
:10B43000C2F878319BE009233B7098E07886FF1FC3
:10B440009194FF1FD895FF1FF495FF1FD894FF1FFD
:10B45000DC95FF1FDD95FF1F0C80FF1F0880FF1F7D
:10B46000008000003893FF1F4A93FF1F9094FF1F36
:10B470004993FF1FCF94FF1F3993FF1FD394FF1FE2
:10B4800001328A4273D03B4850F822409C424FEA36
:10B490008206F5D18319481E824204D25C6843F8C3
:10B4A000044B0132F7E7C5F8740160E0324A00232B
:10B4B000C2F874312F4A002199500433282BF9D156
:10B4C00055E00A237B6052E003233B704FE0737822
:10B4D000812B7EF401ACB278284B922A7EF4FCAB2F
:10B4E0009A79A32A7EF4F8AB5A79B42A7EF4F4ABA5
:10B4F0001A79C52A7EF4F0ABDB78D62B7EF4ECAB60
:10B50000FDF749FBFDF788F80446FDF785F8001BB9
:10B510000028B8BF4042B0F57A7FF6DBFDF758F956
:10B52000174B00221A604FF0FF32C3F87021C3F8A6
:10B530007022C3F87421C3F87422C3F87821C3F8C9
:10B540007822C3F87C21C3F87C220E4B0E4A1A6085
:10B550000120FDF743F90AE040F2D242934206D1BE
:10B56000054B012283F8A02101E00223237004B0DF
:10B57000BDE8F081F087FF1F7886FF1FD094FF1F82
:10B5800010E000E00080FF1F785634123C4B2DE99C
:10B59000F04100241C603B4B3B4E1C603B4BB465B0
:10B5A0001C6086F881402546394B03EB85131A7ED3
:10B5B000384BA3F1100003F10C012AB9364A32517D
:10B5C0001A5102510A5107E0344A3251344A1A5191
:10B5D000344B0351344B0B515FFA85F82721404619
:10B5E00001F08AFD314B1851314B0027EF542621D1
:10B5F000404601F081FD2F4B18512F4B4046EF5430
:10B60000013501F06DFC032D04F10404CCD13B465F
:10B610002A4A002199500433B3F5806FF8D1284F9E
:10B62000BB7E83B10C250024264905F28C60294499
:10B630002044214404220434FDF7C1FB0C2CF3D137
:10B640000C35FC2DEFD1FB7E13B17B7D9BB10DE062
:10B650004FF4FF641C49204621440422FDF7AFFB50
:10B66000043440F6D8039C42F4D1EEE7FDF758FAD3
:10B6700008B1012300E0002386F85430BDE8F081D2
:10B68000D895FF1FF495FF1F7886FF1FD894FF1FE2
:10B690007093FF1FA086FF1FF9D900002DD900006D
:10B6A00091D9000069D90000D1D900008486FF1F1C
:10B6B0004693FF1FC094FF1FCC94FF1FF895FF1FF8
:10B6C0000C80FF1FDC94FF1F008EFF1FF7B50F4C8F
:10B6D0000F4E86460F4694E80300C6F803300D4B24
:10B6E000B27000228DE803001A7086F800E07770CF
:10B6F000FEF7DAF9084A217882F8A1119DE80300E3
:10B70000636884E80300184603B0F0BDEC95FF1FA2
:10B71000D094FF1FE795FF1F7886FF1FF7B51F4ED8
:10B7200002460C4696E803008DE803001C49537856
:10B730000B7093784B70D3788B7013798B7153792E
:10B740004B7193790B71D379CB70164B00271F7017
:10B75000FEF7AAF9144B19786D46334671B921707A
:10B7600061703278A2707278E270F2792271B279E7
:10B7700062717279A2713279E27109E0012907D10F
:10B780003A460A4911444978A1540132082AF8D1AD
:10B7900095E8030083E8030003B0F0BDEC95FF1FBC
:10B7A000D094FF1FE795FF1FDC95FF1FDD95FF1F5E
:10B7B000014B93F8A10170477886FF1F2DE9F043F4
:10B7C000A84BA94C1B788FB063B1A84B1B78062BF4
:10B7D00008D00A2B06D003F0EF030F2B1CBF002369
:10B7E00084F8703194F87031A14E5A1E012A3BD86A
:10B7F000A049012BCA68079214BF082307238DF8BC
:10B800001830327894F8A2318DF8193000238DF871
:10B810001A30C2B98B688DF82030974B8DF82720ED
:10B8200019788DF8211059788DF82210D9798DF872
:10B83000231099798DF8241059791B798DF82510EA
:10B840008DF8263009E0012A07D1013306AA8B4979
:10B850001A44595CD171082BF7D106A801F0A8F958
:10B86000002800F03483A3E0032B1FD133788BB979
:10B87000804F814DB87897F801802A7880449044B1
:10B880006A789044EA799044AA7990446A7990441D
:10B890002A7918E0012B40F08B800025774B585D0A
:10B8A0000135FCF7F3FE092DF8D181E0042B28D1F6
:10B8B000704F714DB87897F80180002301226B70AA
:10B8C0002A706B6080449044FCF7E0FE7878FCF7C7
:10B8D000DDFE2878FCF7DAFE6878FCF7D7FEE87919
:10B8E000FCF7D4FEA879FCF7D1FE6879FCF7CEFE10
:10B8F0005FFA88F82879FCF7C9FE4046FCF7C6FED7
:10B9000056E0072B32D133782BBB5A4B93F802E029
:10B9100093F801C0584B8DF800E01F785D78D87916
:10B920008DF80270E644774499798DF803503D44D0
:10B930005A798DF8040028441B798DF805100144CC
:10B940008DF806200A448DF8073013448DF801C0A5
:10B950008DF8083029E0012B27D10023474A9A5C53
:10B960000DF803200133092BF8D11EE0082B1FD15D
:10B97000414A002301205370107053603D4A8DF8F6
:10B980000200917852788DF801200A4402448DF823
:10B9900000108DF803308DF804308DF805308DF8E7
:10B9A00006308DF807308DF808206846FDF7F0F86E
:10B9B000334B1A789846002A00F08B80314B324D79
:10B9C0001B78013B062B00F28080DFE803F00404C3
:10B9D000257E7E7E5F00274A297893688DF8303077
:10B9E00080238DF831308A238DF8323000238DF892
:10B9F00033308DF834308DF835308DF836108DF8C1
:10BA0000293007218DF82A300AA8D3688DF828102C
:10BA10000B9301F0CDF858E0164F2A78B87897F8D4
:10BA20000190814409F10A099144FCF72FFE7878CE
:10BA3000FCF72CFE8020FCF729FE8A20FCF726FE6E
:10BA40000020FCF723FE0020FCF720FE0020FCF77E
:10BA50001DFE5FFA89F92878FCF718FE4846FCF7C6
:10BA600015FE32E0E695FF1F7886FF1FD094FF1F7A
:10BA7000DC95FF1F0C80FF1FEC95FF1FDD95FF1F5E
:10BA8000CF94FF1F9094FF1F4993FF1F924B2A787A
:10BA9000987859788DF80D10802301448DF80E3078
:10BAA0000A318A238DF80C008DF80F308DF81320A1
:10BAB00000230A4403A88DF810308DF811308DF85A
:10BAC00012308DF81420FDF763F800232B7088F8EE
:10BAD0000030002384F87031337094F8A03113B132
:10BAE0000120FCF77BFE06A800F0EEFF0546A0B3A0
:10BAF0007A4B9DF820201A709DF821205A709DF8ED
:10BB000022209A709DF823209A719DF824205A7162
:10BB10009DF825201A719DF82620DA709DF81930BD
:10BB200084F8A231FCF778FD6D4B6E4D18606E4BBA
:10BB300000221A709DF8183094F85420072B0CBF7F
:10BB40000123022385F87031531E012B674B02D964
:10BB5000052A40F0A0800022BCE003A8FCF7AEFD5F
:10BB6000064600285CD0FCF7C1FD08B184F8A3515B
:10BB700094F8A3119DF80C005A4A4B1CDBB22144E7
:10BB8000092B84F8A33181F8A40140F0B880002388
:10BB900092F8A41182F8A3314F4A5278914240F0B2
:10BBA000AE801A464F4D05F5D271595C01330A44F7
:10BBB000082BD2B2F6D195F8AC3193422CD1474B39
:10BBC00095F8A5211A7095F8A6215A7095F8A72125
:10BBD0009A7095F8A8219A7195F8A9215A7195F84B
:10BBE000AA211A7195F8AB21DA70FCF715FD404BCC
:10BBF000404A186095F8541000231370032285F80A
:10BC000070214A1E012A85F8A331384A02D9052934
:10BC100018BF0123137072E0042385F870316EE0C1
:10BC20000AAD2846FCF7A1FF00283BD03346324638
:10BC3000E95C01330A44082BD2B2F9D19DF83010E7
:10BC400091422CD1254B9DF829201A709DF82A206D
:10BC50005A709DF82B209A709DF82C209A719DF8AF
:10BC60002D205A719DF82E201A719DF82F20DA7020
:10BC7000FCF7D2FC1E4B1F4A1860002313700722EA
:10BC800084F8702194F85420511E01291946174B4D
:10BC900003D9052A01D001221CE019702FE084F895
:10BCA00070312CE094F854300E4D013B012B26D816
:10BCB000AB6DB3F5C05F1FD2FCF732FFE0B1A86DEA
:10BCC0000649431CAB65FDF791F8092385F87031EF
:10BCD000064B01221A7012E00C80FF1FD094FF1F48
:10BCE0008094FF1F7886FF1F2893FF1FE795FF1F93
:10BCF0008894FF1F8F94FF1F002384F8543094F81A
:10BD00005430744D042B04D1734E3278170640F131
:10BD1000B38094F8703113F0FB0F05D0082B03D0DB
:10BD2000062B01D0FDF7C0FE94F87031092B7BD1B2
:10BD3000FCF772FC674A694D926C2B68801A80EAA6
:10BD4000E072A2EBE0729A4208D9654B1A78012A98
:10BD500004BF02221A70FCF75FFCA064FCF75CFCD5
:10BD6000E36C6A68C01A80EAE073A3EBE073934265
:10BD700008D95B4B5A78012A04BF02225A70FCF79B
:10BD80004BFCE064FCF748FC236DAA68C01A80EA0B
:10BD9000E073A3EBE073934208D9514B9A78012AE0
:10BDA00004BF02229A70FCF737FC206594F88030BB
:10BDB000002B39D0474B93F86821002A34D14849E9
:10BDC0008B5C022B2DD1434B03F18C0050F82200E9
:10BDD000451C24D0434983F864210968C3F84811FD
:10BDE00041490968C3F84C11996DC3F850113F4996
:10BDF00098650968C3F8541193F88110C3F8581175
:10BE00000022D3F88810C3F85C1183F88120D3F89E
:10BE10008410C3F86011012283F8682104E0002334
:10BE20008B5401322F2ACAD194F87011294B092959
:10BE300006D193F85420022A04BF052283F8542027
:10BE4000D4F87421234B002A41D009293FD193F81B
:10BE5000541001293BD1986D00231E4901F5BC7493
:10BE600054F82340A04203D1052381F854302EE03A
:10BE700001339342F1D12AE095F8703113F0FB0FB2
:10BE800025D0082B23D0062B21D0D5F86C01184CD7
:10BE9000D6F803306270B0F5C05F636012D23146ED
:10BEA000FCF79DFFD5F86C013146FCF7C3FF30B1BC
:10BEB000D5F86C310133C5F86C31652300E00723F8
:10BEC000237004E007232370002385F854300FB05B
:10BED000BDE8F0837886FF1FD094FF1F4094FF1FBA
:10BEE0009194FF1FD895FF1FF495FF1FD894FF1F53
:10BEF000EC95FF1FAFF30080704710B5074CFCF7BF
:10BF00008BFB2368C01AB0F5FA7F05D9044B0222D7
:10BF1000DA60FCF781FB206010BD00BFF899FF1FBD
:10BF200000F00F40704708B5034B5878FCF7A2FDAE
:10BF3000024B586008BD00BFD094FF1FEC95FF1F57
:10BF40007047704770477047704708B5034B3B21F7
:10BF5000987801F0D1F8024B586008BDD094FF1FCB
:10BF6000EC95FF1F00000000014B53F820007047C4
:10BF70002888FF1F2DE9F0479B4DEB69C3B19B4C0F
:10BF80002678AEB9FCF748FB994B1B68C01AEB69E1
:10BF90000028B8BF404298420AD9304601F08EFCD2
:10BFA000012001F08BFC022001F088FC01232370AA
:10BFB0002B6AD3B18F4C2578BDB9FCF72DFB8E4B86
:10BFC000894A1B68126AC01A80EAE073A3EBE07327
:10BFD00093420AD9284601F071FC012001F06EFC61
:10BFE000022001F06BFC01232370844CFCF714FB4E
:10BFF000237E04EB8303DB68C01A80EAE073A3EBC3
:10C00000E0730A2B25DDFCF707FB21210646207E85
:10C0100001F072F894F8188004EB88050746E86987
:10C02000381A04F011FA8146E868301A04F00CFA64
:10C030000146484604F010FB03F036FE68A3D3E93E
:10C04000002303F085FE04F01DF944F82800EE609B
:10C05000EF61207E694E352101F04EF810F0400965
:10C0600005460DD0307E01F029FC337E644A012163
:10C07000D1540F33634AD15C012904BF0221D1544A
:10C08000614B207E5D4E03EB801298461269FAB137
:10C09000222101F031F8377E08EB87130028B8BF62
:10C0A00040421B69984213D9F31993F8283023BBF7
:10C0B0003421384601F020F8342140F480623846BB
:10C0C00000F0EAFF337E1E44012386F8283014E096
:10C0D000267E4A4FA31993F8283073B13421304695
:10C0E00001F00AF8342120F48062304600F0D4FFD9
:10C0F0003B7E1F44002387F8283094F82B60DFF83C
:10C100000CA15EB9F0B2FCF766FC0AF80600013635
:10C11000082EF7D1394B012283F82B202726002740
:10C12000F8B2FCF758FC1AF8073083421BD0374BA3
:10C1300007F10802F854364B53F82230022B05D091
:10C14000032B0AD0012B0ED168B106E058B92D4A55
:10C15000915D012907D1935505E02A4B9A5D012A8B
:10C1600004BF02229A550137082F06F10106D7D1E4
:10C17000237E15F0010104EB03020BD092F834107A
:10C18000E1B9012182F83410214A1A44127E12F0DA
:10C19000010F09E092F8340080B182F834101C4A93
:10C1A0001A44127E12F0020F08D002211B2211FB4A
:10C1B0000323144AD05C012808BFD154237EE2181F
:10C1C000AE0792F8371025D5002936D1012182F823
:10C1D00037100F4A1A44D27E12F0010F23E000BF3D
:10C1E000FCA9F1D24D6290400C80FF1F8F94FF1F7D
:10C1F0008894FF1F2893FF1F8094FF1F2888FF1F2C
:10C200006893FF1F9194FF1F7093FF1F5488FF1FB7
:10C210004094FF1F89B1012182F83710384A1A442F
:10C22000D27E12F0020F08D00E33364A12F81310E5
:10C23000012904BF022102F8131015F0800107D074
:10C24000237E304A0333D05C012804BF0220D0543F
:10C25000B9F1000F07D0237E2A4A0F33D05C0128A2
:10C2600004BF0220D05499B1274B217E1A7842FA9C
:10C2700001F0C0070CD50120244E00FA01F1317005
:10C28000234E30702348007810B922EA01021A7058
:10C29000207E214E08EB80131B6A1BB36B0521D453
:10C2A000392100F029FF21210546307E00F024FFCE
:10C2B000337E1A4A02EB8312281A126A80EAE0756A
:10C2C000A5EBE07595420DD9184601F0F7FA337EDB
:10C2D000134A0121D15415330A4AD15C012904BF04
:10C2E0000221D154207E0C4D00F04CF8237E013306
:10C2F000DBB2022B88BF00232B76BDE8F08700BF9E
:10C300004094FF1F9194FF1F4A93FF1F4993FF1F03
:10C31000CF94FF1F3893FF1F2888FF1F7093FF1FC4
:10C320004393FF1FAFF3008073B5134E335C044695
:10C330000D463BB1114B262153F8202000F0ACFEF6
:10C340000023335585EAE572A2EBE57220462721EA
:10C3500000F0A2FE0A4A0123002D13554FF00002FF
:10C36000D8BF02230193009220462021134600F0FB
:10C3700057FE02B070BD00BFCC94FF1FC094FF1FDA
:10C380004693FF1F2DE9F04F352185B0044600F09C
:10C39000B3FE8346A948A10146184FEA5B03327AEF
:10C3A000766812F0400F0BF0010508D0415803F0F9
:10C3B0000107C1F1000AEBB2C6F1000905E050F82F
:10C3C00001A0EFB203F00103B1460393130602F09C
:10C3D0003F06204607D501F091FAD0F1010838BF99
:10C3E0004FF0000806E001F089FA10F1000818BFCC
:10C3F0004FF00108721E039B072A00F20A82DFE851
:10C4000012F00800080008000800E900E900E9004F
:10C41000E9008B4D2A5D013A0E2A00F2FA81DFE82D
:10C4200012F00F0021002500300034003C004A00CB
:10C4300058008700A900AD00F801D400EF01E90120
:10C440003421204600F058FE05EB84057D4A7C4BE4
:10C4500068600121023E8E42115594BF02220422DF
:10C460001A55D6E105EB84035A68E2E0002B00F090
:10C47000D0812046212100F03FFE734B43F8240079
:10C48000FDE005EB84035A6808E1002F00F0C1814C
:10C49000204601F013FA0623BAE105EB8403204697
:10C4A0005A68342122F0030200F0F6FD2046494686
:10C4B000FFF73AFF17E1002F40F0AB8120463946E5
:10C4C000FFF732FF2046C9F10001FFF72DFF0823D7
:10C4D0009EE1002F00F09D812121204600F00CFEFE
:10C4E000002106462046FFF71FFF574B53F8242034
:10C4F000921B43F8242005EB840320465A6834211C
:10C5000022F0030200F0C8FD204627214A4600F031
:10C51000C3FD20462D21324600F0BEFD0022134609
:10C52000009201922046202100F07AFD09236FE15C
:10C530001BF4007F00F06D812121204600F0DCFD1E
:10C54000424B002118602046FFF7EEFE20462D21C9
:10C55000002200F0A1FD20462121002200F09CFDD8
:10C56000033E20463921002200F096FD012E00F204
:10C570004581E0E0002F00F04C81EDE0002F40F01D
:10C5800048812121204600F0B7FD39460646204665
:10C59000FFF7CAFE05EB840320465A68342122F0D7
:10C5A000030200F079FD204627214A4600F074FD81
:10C5B000022220462D2196FBF2F200F06DFD00973D
:10C5C0000197204620213A46EEE01BF4007F00F060
:10C5D000208113E11A4D2A5D013A0E2A00F21981D9
:10C5E000DFE812F00F00200047005500730017012C
:10C5F000830017011701B000BC009800E7000E018E
:10C600000801104B0122204634211A5500F074FD18
:10C6100005EB8403062E58605DD0082E5BD0042203
:10C62000074B1DE7062E13D105EB84035A6822F051
:10C6300003022046342142F0020212E07093FF1FF1
:10C640006488FF1F4693FF1F2C93FF1F3494FF1F26
:10C65000082E08D105EB840320465A68342122F0C5
:10C66000030200F019FD20465146FFF75DFE03234B
:10C67000CEE0721F012A04D81BB1062E2DD104234F
:10C68000C6E0B8F1000F00F0C4800C23C0E0052E16
:10C6900009D105EB84035A6822F0030220463421B5
:10C6A00042F0010208E0072E08D105EB8403204682
:10C6B0005A68342122F0030200F0EEFC2046CAF151
:10C6C0000001FFF731FE0523A2E0731F012B06D8FE
:10C6D0002FB1052E01D102239AE00F2398E0B8F183
:10C6E000000F00F09680072392E0B8F1000F40F0B1
:10C6F0009080073E012E0AD905EB840320465A6834
:10C7000022F00302342142F0020200F0C5FC204670
:10C71000494613E0B8F1000F7BD1073E012E0AD93C
:10C7200005EB840320465A6822F00302342142F0CC
:10C73000010200F0B1FC2046C9F10001FFF7F4FD51
:10C740000A2365E0B8F1000F63D02046212100F0F4
:10C75000D3FC05EB840318610B2359E0B8F1000FFB
:10C7600057D1212105EB8406204600F0C5FC7268F4
:10C7700007463421204622F0030200F08DFC2046BB
:10C7800027214A4600F088FC336902221F442046D4
:10C790002D2197FBF2F200F07FFCCDF80080CDF860
:10C7A0000480204620214246134600F039FC0D2328
:10C7B0002EE01BF4007F2CD00E23204621212B5588
:10C7C00000F09AFC144B002118602046FFF7ACFDE6
:10C7D00020462D21002200F05FFC2046212100226E
:10C7E00000F05AFC20463921002205B0BDE8F04F88
:10C7F00000F052BC20460021FFF796FD0E2307E013
:10C8000005EB840320465A68342100F045FC0023E0
:10C810002B5505B0BDE8F08F3494FF1F024B1A5C16
:10C820000AB901221A5470476488FF1F024B1A5C30
:10C830000AB10F221A5470476488FF1F014B185C1D
:10C84000704700BF6488FF1F104A684620F0070148
:10C8500013698D4640F273214B434FF6FF71B3FBD2
:10C86000F1F36E2B01B504D9094B4FF480215960C7
:10C8700005E04F2B03D8064B4FF480219960BDE8AB
:10C880000140572313608546704700BF00B0034046
:10C8900080F00F401F4B68461A6820F007018D4654
:10C8A00002F01F0201B5072A2DD8DFE802F0040AC2
:10C8B0002C10161C22281969174A89B211804122AE
:10C8C00022E01969144A89B2518043221CE0196997
:10C8D000114A89B2D180442216E019690E4A89B200
:10C8E0001181452210E019690B4A89B25181462213
:10C8F0000AE01969084A89B29181472204E019695E
:10C90000054A89B2D1814022BDE801401A608546BE
:10C91000704700BF00B00B408088FF1F38B541F260
:10C920003002114B995841F00061995041F23C029C
:10C930000024995841F00061995003F5E8230D2532
:10C9400040229D604920DC605C621A6001F070F852
:10C95000064B57229D602720DC605C621A60BDE8B0
:10C96000384001F065B800BF0070044000B00340DB
:10C970000B2829D8DFE800F006090D102828282800
:10C980001328191E114B188901E0104B588980B2E9
:10C9900070470E4B9889FAE70C4BD889F7E70B4B99
:10C9A000588840F2732380B208E0084BD8888E2361
:10C9B00080B203E0054B1888422380B258434FF6FB
:10C9C000FF7390FBF3F07047002070478088FF1FD3
:10C9D00030B541F23C032E4CE55845F01005E550CA
:10C9E0002C4B4FF400741C636FF4F8755C63A3F573
:10C9F0001433A4F13E542C441C604FF400545C608A
:10CA0000254C1C601C68E401FCD50138072813D8AC
:10CA1000DFE800F0100E0C0A081206041F480CE0B4
:10CA20001F480AE01F4808E01F4806E01F4804E0CE
:10CA30001F4802E01F4800E01F4858601F4B0020BD
:10CA400058631F4818601F488D044FF080642840C9
:10CA5000C3F88040C3F884003AB11A48C3F8904044
:10CA600094042040C3F8940001E0C3F890204FF0F4
:10CA70008464C3F8A0401148C3F8A41022B1C0F8E0
:10CA8000B040C0F8B42030BDC0F8B02030BD00BF09
:10CA900000700440009004400F0080508720FE0189
:10CAA0008720FE038720FE0F8720FE138720FE27A6
:10CAB0008720FE638720FEC78720FE0700400240D4
:10CAC0000F0080000000FC1F384BD3F88020C2F319
:10CAD0000362022A10B513D0D3F89020C2F3036288
:10CAE000022A0FD0D3F8A020C2F30362022A0AD090
:10CAF000D3F8B030C3F30363022B54D1032202E016
:10CB0000002200E00122120102F1402303F500336C
:10CB1000D3F88010C1F303410170D3F8801011F4F1
:10CB2000801118BF01218170D3F8801011F4001119
:10CB300018BF01214170417821B9D3F88410C1F3A5
:10CB40008A4103E0D3F8841021F0604102F14022D1
:10CB500002F500324160D2F88840240E0472D2F807
:10CB60008840240C4472D2F88840240A847202F16E
:10CB70008801D2F88820C2724A68120E02734A688D
:10CB8000120C42734A68120A82734A68C273D3F85D
:10CB9000802092024CBF4FF084624FF08062C3F855
:10CBA0008020012010BD002010BD00BF00400240C9
:10CBB000204BD3F87021C2F303620C2A38D041789D
:10CBC000426811B1C2F3110202E091041A4A0A400C
:10CBD000C3F87421427A037A120442EA0362C37AE8
:10CBE0001A43837A42EA0322124BC3F87821427B2C
:10CBF000017B120442EA0162C17B0A43817B42EA63
:10CC00000122C3F87C2143788278002B14BF4FF0B7
:10CC100042634FF040630AB143F480130278120478
:10CC200002F470221343034A0120C2F870317047A6
:10CC300000207047004002400000FC1F0B4B4FF0EB
:10CC40000062C3F870214FF48022C3F87421084AAF
:10CC5000C3F878216FF48471A2F166320A44C3F8F4
:10CC60007C21044AC3F87021704700BF0040024095
:10CC7000785634120000080C684620F007018D46F3
:10CC800011B53D4BDA7842F00202DA703B4A107877
:10CC9000C0B20228114641D0032835D0012867D1FF
:10CCA000547891788C4216D2D978C90709D4517832
:10CCB0005068C9B24C1CE4B25470425CD2B21A71D2
:10CCC00056E0997801F0DF019970997801F0EF0151
:10CCD000997010724AE0517A01F0FF0049B99978D1
:10CCE00001F0DF019970997801F0EF0199701070EF
:10CCF0003EE0997841F004019970917AC9B21971B6
:10CD000000235372032332E0997801F0EF01997008
:10CD10001B79D168DBB20B70022328E0147C507CB5
:10CD200084421FD2507C127C821A012A05D19A7843
:10CD300002F0DF029A7000230B704A7C0B7CD31A3E
:10CD4000022B04DC0C4B9A7842F008029A700B7CA0
:10CD5000CA68DBB2581CC0B2087407490979C9B265
:10CD6000D15405E0997801F0DF0199700023137028
:10CD7000BDE8114085467047007006409088FF1F4F
:10CD80000B4A41F234031920D15841F08001D150AF
:10CD9000084B4FF400729A62DA6203F5E0331B220B
:10CDA0005A70C0229A7000225A7100F041BE00BF32
:10CDB0000070044000B0044010B5124B0024D2B201
:10CDC0001C725C729A7001225C701A700E4A596073
:10CDD000917801F0F7019170917841F01001917014
:10CDE000917800F0FE0041F02001917010711A78E6
:10CDF000002AFCD1034B187AD0F1010038BF002083
:10CE000010BD00BF9088FF1F0070064010B5124B88
:10CE10000024D2B21C725C725A7403221C741A7001
:10CE20000E4AD960917801F0F7019170917841F044
:10CE300010019170917840F0010041F02001917053
:10CE400010711A78002AFCD1034B187AD0F1010036
:10CE500038BF002010BD00BF9088FF1F0070064043
:10CE600070B5164C0025E36001269DF81030257240
:10CE7000D2B26672A2706570637440EA06032574CC
:10CE8000A3720F4B616026709A7802F0F7029A70D5
:10CE90009A7842F010029A709A7800F0FE0042F000
:10CEA00020029A7018712378002BFCD1034B187A5A
:10CEB000D0F1010038BF002070BD00BF9088FF1F77
:10CEC000007006400000000010B50024E0B23A21D6
:10CED0004FF48032013400F0DFF8032CF6D110BD9E
:10CEE0002DE9F743484C04EB8014183463688046FE
:10CEF0000BB1658875B93821404600F0FDF838213E
:10CF000020F48062404600F0C7F840463A214FF4D2
:10CF1000803270E000F092FAC0F1080005FA00F0EB
:10CF200002F0B0FED4F80490044689EAE970A0EB60
:10CF3000E9700D4602F0A6FE02460B462046294641
:10CF400003F030F8314B002204460D4602F000FF9A
:10CF50006A4606460F4603F0DFFC0022002303F07A
:10CF60005FF980B13946304603F08CF9B9F1000F12
:10CF700004464FF03801B8BF4442404600F0BCF8C8
:10CF800020F4806230E0204629466A4603F0C4FC63
:10CF9000B9F1000F04460D46DDE900010CDD03F098
:10CFA00071F917A3D3E9002306042946204602F0AD
:10CFB000CFFE03F067F90FE003F064F9C04310A35C
:10CFC000D3E9002306042946204602F0C1FE03F0FF
:10CFD00059F9C0F51C50103040EA0604382140468B
:10CFE00000F08AF840F480624046382100F054F89E
:10CFF00040463A21224603B0BDE8F04300F04CB869
:10D00000000000000088C3407093FF1F0000F04044
:10D01000392100F071B80A46392100F03DB800BF4F
:10D020002DE9F0471F461A4B9DF8206033F8104059
:10D030009DF82450904681468A46002241F08001A6
:10D040002046FBF7FDFD414600222046FBF7F8FD98
:10D05000394600222046FBF7F3FD0AF07F0A3146ED
:10D0600000222046FBF7ECFD47EA08272946204628
:10D0700001220AEB4A0AFBF7E3FD46EA0726D14400
:10D08000044B45EA062543F82950BDE8F08700BF68
:10D09000680D0100A488FF1FF8B5154B33F8105038
:10D0A000144606460F46002241F080012846FBF751
:10D0B000C7FD210E00222846FBF7C2FDC4F307413D
:10D0C00000222846FBF7BCFD07F07F07C4F30721C9
:10D0D00000222846FBF7B4FD07EB47072846E1B2DC
:10D0E0000122FBF7ADFD3E44024B43F82640F8BD5C
:10D0F000680D0100A488FF1F294B70B501F07F0562
:10D100005A19127B002A43D033F8104029460022D6
:10D110002046FBF795FD00210A462046FBF790FDCF
:10D1200000210A462046FBF78BFD00210A462046D7
:10D13000FBF786FD002101222046FBF781FD00213F
:10D140000A462046FBF77CFD00210A462046FBF7F5
:10D1500077FD002106020A462046FBF771FD0021FB
:10D16000304306020A462046FBF76AFD30430602BA
:10D17000002120460122FBF763FD222D46EA000034
:10D1800001D0422D0AD1030208D540F07F4070BD86
:10D1900005EB45052844034B53F8200070BD00BF44
:10D1A000680D0100A488FF1F70B50B4C04440646AF
:10D1B00094F800360D465BB96C21FFF79DFF05F032
:10D1C0000F0320F00F026C2130461A43FFF764FF73
:10D1D00084F8035670BD00BFA488FF1F38B50D4604
:10D1E0006C210446FFF788FF05F0070220F070036A
:10D1F00043EA021220466C21BDE83840FFF74CBFDD
:10D2000038B50D466C210446FFF776FF05F00F0296
:10D2100020F4F06343EAC21220466C21BDE8384096
:10D22000FFF73ABF38B50D466C210446FFF764FF9F
:10D2300005F0030220F4C03343EAC23220466C21D9
:10D24000BDE83840FFF728BF38B50D466C210446CD
:10D25000FFF752FF05F00F0220F4700343EA025279
:10D2600020466C21BDE83840FFF716BF38B50D46A3
:10D270006C210446FFF740FF05F00F0220F07063B9
:10D2800043EA026220466C21BDE83840FFF704BF44
:10D2900038B50C466C210546FFF72EFF14B140F05F
:10D2A000804201E020F0804228466C21BDE83840F1
:10D2B000FFF7F2BE38B50C466C210546FFF71CFFA0
:10D2C00014B140F4002201E020F4002228466C2131
:10D2D000BDE83840FFF7E0BE38B50C466C21054686
:10D2E000FFF70AFF14B140F4802201E020F480220D
:10D2F00028466C21BDE83840FFF7CEBE38B50C4655
:10D300006C210546FFF7F8FE14B140F4804201E0BD
:10D3100020F4804228466C21BDE83840FFF7BCBEAF
:10D3200038B50C466C210546FFF7E6FE14B140F413
:10D33000005201E020F4005228466C21BDE838403C
:10D34000FFF7AABE38B50C466C210546FFF7D4FEA0
:10D3500014B140F4805201E020F4805228466C2140
:10D36000BDE83840FFF798BE38B50C466C2105463D
:10D37000FFF7C2FE23074ABF20F0700320F40763C3
:10D3800043F4006304F00702284643EA02126C21CA
:10D39000BDE83840FFF780BE38B50D466C21044625
:10D3A000FFF7AAFE05F00F0220F4F06343EAC21271
:10D3B00020466C21BDE83840FFF76EBE38B50C46FC
:10D3C0006C210546FFF798FE14B140F4003201E0ED
:10D3D00020F4003228466C21BDE83840FFF75CBEDF
:10D3E00008B5074B034493F800262AB96C21FFF7D0
:10D3F00083FE00F00F0008BD93F8030608BD00BFD0
:10D40000A488FF1F08B56C21FFF776FEC0F3021059
:10D4100008BD08B56C21FFF76FFEC0F3C31008BD4F
:10D4200008B56C21FFF768FEC0F3C13008BD08B530
:10D430006C21FFF761FEC0F3035008BD08B56C21F5
:10D44000FFF75AFEC0F3036008BD08B56C21FFF773
:10D4500053FEC0F3807008BD08B56C21FFF74CFE89
:10D46000C0F3C04008BD08B56C21FFF745FEC0F30E
:10D47000804008BD08B56C21FFF73EFEC0F3803048
:10D4800008BD08B56C21FFF737FEC0F3403008BD7A
:10D4900008B56C21FFF730FEC0F3003008BD08B5B9
:10D4A0006C21FFF729FEC0F30213020548BF43F0C9
:10D4B0000803184608BD08B56C21FFF71DFEC0F330
:10D4C000C31008BD08B56C21FFF716FEC0F340403D
:10D4D00008BD38B50D466D210446FFF70DFE05F079
:10D4E000030220F0600343EA421220466D21BDE8AA
:10D4F0003840FFF7D1BD38B50D466D210446FFF722
:10D50000FBFD05F0030220F4C04343EA423220460B
:10D510006D21BDE83840FFF7BFBD38B50D466D2120
:10D520000446FFF7E9FD05F00F0220F4706343EABB
:10D53000022220466D21BDE83840FFF7ADBD38B569
:10D540000D466D210446FFF7D7FD05F00F0320F0CF
:10D550000F021A4320466D21BDE83840FFF79CBDFD
:10D5600038B50C466D210546FFF7C6FD20F47F0255
:10D5700042EA044228466D21BDE83840FFF78CBDE1
:10D5800038B50C466D210546FFF7B6FD14B140F4E1
:10D59000004201E020F4004228466D21BDE83840F9
:10D5A000FFF77ABD38B50C466D210546FFF7A4FD9F
:10D5B00014B140F0807201E020F0807228466D21A5
:10D5C000BDE83840FFF768BD08B56D21FFF794FD51
:10D5D000C0F3411008BD08B56D21FFF78DFDC0F304
:10D5E000413008BD08B56D21FFF786FDC0F303206B
:10D5F00008BD08B56D21FFF77FFD00F00F0008BDE5
:10D6000008B56D21FFF778FD0314D8B21B0648BF9B
:10D6100060F0FF0008BD08B56D21FFF76DFDC0F398
:10D62000C03008BD08B56D21FFF766FDC0F300608E
:10D6300008BD38B50D4670210446FFF75DFD05F0C5
:10D64000030220F4401343EA025220467021BDE851
:10D650003840FFF721BD38B50C4670210546FFF76D
:10D660004BFD14B140F4002201E020F400222846D2
:10D670007021BDE83840FFF70FBD38B50C4670216A
:10D680000546FFF739FD14B140F4802201E020F493
:10D69000802228467021BDE83840FFF7FDBC38B530
:10D6A0000D4670210446FFF727FD05F0030220F424
:10D6B000403343EA024220467021BDE83840FFF77C
:10D6C000EBBC38B50C4670210546FFF715FD20F47C
:10D6D0007F4242EA042228467021BDE83840FFF725
:10D6E000DBBC38B50C4670210546FFF705FD20F080
:10D6F000FF02224328467021BDE83840FFF7CCBC2A
:10D7000008B57021FFF7F8FCC0F3015008BD08B55B
:10D710007021FFF7F1FCC0F3C04008BD08B57021CF
:10D72000FFF7EAFCC0F3804008BD08B57021FFF7A1
:10D73000E3FCC0F3014008BD08B57021FFF7DCFC35
:10D74000C0F3072008BD08B57021FFF7D5FCC0B2B3
:10D7500008BD70B50C466F2115461E46FFF7CCFC80
:10D7600014B1C0F34923236015B1C0F304432B70F7
:10D770000EB1000E307070BDF7B5FAF74DFF0446DC
:10D78000FAF74AFF001B0028B8BF40420928F7DD1E
:10D790000025ECB200210A462046FFF77DFC02225C
:10D7A00055238DE80C0020466C2100220123FFF751
:10D7B00037FC01270F238DE888002046072310211E
:10D7C0000022FFF72DFC7021284A2046FFF764FC59
:10D7D0002046FFF705FE264B5855033B0026EE5426
:10D7E000204620213246FFF757FC20462D213246A5
:10D7F000FFF752FC204621213246FFF74DFC204620
:10D8000023213A46FFF748FC20462421DC22FFF77B
:10D8100043FC2046252146F6DB02FFF73DFC20466F
:10D82000262140F2B712FFF737FC204627214DF2A0
:10D83000B712FFF731FC2046282140F2B712FFF75C
:10D840002BFC20462A21DC22FFF726FC20462B2138
:10D850000A22FFF721FC3D4420461421054AFFF728
:10D860001BFC032D95D103B0F0BD00BF8004050063
:10D87000A78EFF1FFFFF0F0038B5074C044494F834
:10D88000001641B994F80356FFF78EFC012384F883
:10D89000003684F8035638BDA488FF1F064B0344A6
:10D8A00093F8002632B1002293F8031683F800267D
:10D8B000FFF77ABC704700BFA488FF1F0D4B37B538
:10D8C00001251D540C4BC4B21D54272120460022B3
:10D8D000FFF7E2FB204626214FF6FF72FFF7DCFB45
:10D8E00000228DE82400204620211346FFF798FBF4
:10D8F00003B030BD4693FF1FCC94FF1F01280CD00E
:10D9000006D302280ED1084B1869C0F300507047A7
:10D91000054B1869C0F380507047034B1869C0F37A
:10D92000405070470020704740F00F40002808B575
:10D9300009DB02F0A7F90AA3D3E9002302F032FBC6
:10D9400003F04AF908E002F09DF905A3D3E90023AA
:10D9500002F028FB03F0B0F802F094FC08BD00BF11
:10D9600034F7FFFF7F84EE3F08B502F08BF906A382
:10D97000D3E9002302F016FB03F02EF902F082FC3B
:10D9800008BD00BFAFF30080EB1100A2941A5D4008
:10D99000002808B509DB02F075F90BA3D3E90023D1
:10D9A00002F0D6F903F088F808E002F06BF906A35C
:10D9B000D3E9002302F0CCF903F00EF902F062FC87
:10D9C00008BD00BFAFF3008034F7FFFF7F84EE3F58
:10D9D00008B502F039FD02F067F905A3D3E9002389
:10D9E00002F0B6F903F068F802F04CFC08BD00BF85
:10D9F000EB1100A2941A5D40704700BFAFF30080A6
:10DA0000FEE74FF0E023084AC3F8082D074A4CF21E
:10DA10002053D3814DF62813D381138823F00103BB
:10DA20001B041B0C13807047008000000020054081
:10DA3000802810B54FF00101154A06DD00F01F00E7
:10DA40008140C2F88C11D16010BD402806DD00F085
:10DA50001F008140C2F88811916010BD20280C463B
:10DA600006DD00F01F008140C2F88411516010BD36
:10DA7000084B0340002B03DA013B63F01F03013323
:10DA8000034A04FA03F3C2F88031136010BD00BFEB
:10DA900000E100E01F000080802810B54FF0010277
:10DAA000134905DD00F01F008240C1F88C2010BD35
:10DAB000402805DD00F01F008240C1F8882010BD1D
:10DAC0002028144605DD00F01F008240C1F88420A4
:10DAD00010BD084B0340002B03DA013B63F01F032A
:10DAE0000133034A04FA03F3C2F8803010BD00BFCB
:10DAF00000E100E01F00008003291ADC202818DC68
:10DB000004220C4B90FBF2F2D2B2034002F16042CD
:10DB10008901002B02F56442C9B203DA013B63F0CC
:10DB200003030133DBB21068DB0001FA03F318438F
:10DB30001060704703000080064B1A78D2B2012AA9
:10DB400005D1222902D0212901D100225A700122B7
:10DB50005A707047AC8EFF1F70B5144611B91B4B3D
:10DB6000197070BD022903D1184B01221A7070BDC3
:10DB7000042914D1154B5B78012B25D195880023FE
:10DB8000402D28BF40255E1CDBB2AB4205D2226887
:10DB9000D05C00F0C7F83346F5E7002007E0032922
:10DBA0000CD10A4B5A78012A0ED10020987002211C
:10DBB00002460346BDE8704000F046BF052903D188
:10DBC000024B00221A705A7070BD00BFAC8EFF1F4E
:10DBD00010B50446204600F0BDF80028FAD110BD6B
:10DBE000704710B5084C02460B4600200121A17079
:10DBF00000F0EEFA224618B10023A370122010BDE7
:10DC00009378002BFCD110BDAC8EFF1FF8B50646F3
:10DC10000F4600F0FAFC0E4B1A78012A16D15B78F9
:10DC2000012B13D100F000F988B10025ECB2BC4201
:10DC300005D330462146BDE8F840FFF7D2BF301982
:10DC400000F0D6F801350028F0D0F2E70C20F8BD3E
:10DC5000AC8EFF1F08B540210248FFF7D7FF00F048
:10DC600095F808BDAF8EFF1F38B5054600F0A8F83F
:10DC70000B28044609D106484021FFF7C7FF28B901
:10DC80002846BDE8384000F09BB80024204638BD47
:10DC9000EF8EFF1FF8B5002406460F462546A3B2B7
:10DCA0009F4207D0305DFFF7DFFF002818BF0B252C
:10DCB0000134F4E72846F8BD38B5451E002415F8B0
:10DCC000010F28B1FFF7D0FF002818BF0B24F6E79B
:10DCD000204638BD07B50123002000930549064BB7
:10DCE000024600F01FFA002814BF1B20002003B0DA
:10DCF0005DF804FB59DB000039DB000038B50D4648
:10DD0000044600F097F885420AD825440020AC422A
:10DD100007D020B914F8010B00F052F8F7E738BD2E
:10DD20000B2038BD10B50A4B197840290ED05A780F
:10DD30009C180132D2B2402AA07001F101014FF0CB
:10DD40000000197014BF5A70587010BD0B2010BD20
:10DD50002F8FFF1F10B50C4B197891B193F842200B
:10DD60009C180132D2B2A4780470402A4FF000000F
:10DD700001F1FF31197014BF83F8422083F842008B
:10DD800010BD0A2010BD00BF2F8FFF1F014B187858
:10DD9000704700BF2F8FFF1F024B1878C0F1400063
:10DDA000C0B270472F8FFF1F034B00225A7083F8B9
:10DDB00042201A70704700BF2F8FFF1FFFF7F4BF7C
:10DDC00010B50A4B197840290ED05A789C180132A8
:10DDD000D2B2402AA07001F101014FF00000197089
:10DDE00014BF5A70587010BD0B2010BD728FFF1FEA
:10DDF00010B50C4B197891B193F842209C18013260
:10DE0000D2B2A4780470402A4FF0000001F1FF3133
:10DE1000197014BF83F8422083F8420010BD0A2015
:10DE200010BD00BF728FFF1F014B1878704700BFF5
:10DE3000728FFF1F024B1878C0F14000C0B27047CC
:10DE4000728FFF1F034B00225A7083F842201A7012
:10DE5000704700BF728FFF1FFFF7F4BF70B5044615
:10DE6000007801F08DF901780023DAB28A4208D2F5
:10DE700003EB8305054466786D78AE4203F1010338
:10DE8000F3D1154D207A342303FB0253D97810B90E
:10DE900098780130987034235A43AB189B788B42A2
:10DEA0000DD003F003030C2101FB03220A4B1A449B
:10DEB000131D107951791B89926800F091FBD5F8F8
:10DEC0009C3043B1227A002A224614BF0521032147
:10DED00012F8080B984770BDB88FFF1F2DE9FF4758
:10DEE0000D4691468DF80F0001F04AF9022D0646C5
:10DEF00049D190F800A00024E3B2534504F1010495
:10DF000009DA03EB830333440DF10F005978DA7813
:10DF100001F0F6F9F0E74FF000085FFA88F757458F
:10DF200027DA07EB870737447C1C6078A378797879
:10DF3000B4F803200090002001900DF10F0001F0D3
:10DF4000BDF96378032B05D19DF80F007978184A45
:10DF500001F03CFA7978A37841F0100141EAC3114D
:10DF60000DF10F00C9B2002201F0FAF908F1010821
:10DF7000D3E7104BD3F89C30B3B19DF80F0029467E
:10DF80004A46984710E0002DF3D12B463278591CB1
:10DF9000DBB29A42EDD9074A342000FB032300226A
:10DFA0009A70DA700B46F1E704B0BDE8F08700BF65
:10DFB0005DDE0000B88FFF1F2DE9F0410C7804F002
:10DFC0006004202C1D4638D14C78042C1CD00AD873
:10DFD000012C2ED02DD3022C1FD0032C29D1BDE82B
:10DFE000F04100F05FB9212C1BD005D8202C20D1A6
:10DFF000BDE8F04100F03EB9222C16D0232C18D1F8
:10E00000BDE8F04100F046B902241C8014680025E8
:10E0100025701468671C17606570BDE8F04100F05A
:10E020005BB9BDE8F04100F01DB9BDE8F04100F07A
:10E030007BB900202880BDE8F081402C06D1054C3A
:10E04000D4F8A04014B1A047BDE8F081CD20BDE8D0
:10E05000F08100BFB88FFF1F73B50446007801F050
:10E060008FF863680093A27A637A43EA0223ADF8DB
:10E07000043001780023DAB28A4208D203EB830528
:10E08000054466786D78AE4203F10103F3D1164D75
:10E09000207A342303FB0253D97810B998780130E1
:10E0A000987034235A43AB189B788B420DD003F001
:10E0B00003030C2101FB03220B4B1A44131D10799F
:10E0C00051791B89926800F08BFAD5F89C304BB1DE
:10E0D000227A20781AB1052104F1080201E0032117
:10E0E0006A46984702B070BDB88FFF1F07B54368F6
:10E0F0000093437A817A43EA0123ADF80430084B58
:10E10000D3F89C30024643B1017A007811B1052161
:10E11000083201E004216A46984703B05DF804FB29
:10E12000B88FFF1F2DE9F8430546884617469946E4
:10E1300001F026F802789DF82030013206460021D1
:10E140002846D2B201F09CF8044630BB2846144958
:10E15000144A00F08EF93378601CE4B2A34211D95E
:10E1600004EB8402324434235C430F4992F801E00B
:10E1700001F804E00B1992785A7000229A70DA7054
:10E180000446E8E72846494600F066F8044620B908
:10E19000054BC3F89C80C3F8A0702046BDE8F88307
:10E1A000DDDE0000B9DF0000B88FFF1F08B5074BA8
:10E1B0000022C3F89C20C3F8A02000F0ADF918B9E4
:10E1C000BDE8084001F072B808BD00BFB88FFF1F5E
:10E1D0002DE9F047914607460D46984600F0D0FFDE
:10E1E00002780024E3B2934207D2013404EB8401A5
:10E1F000014411F8041CA942F4D1164A34205843B2
:10E200001118CE788B78F41AE4B2042C02D1C12014
:10E21000BDE8F08706F003044FF00C0C0CFB04047F
:10E2200014440136F6B227716571C4F80890A4F859
:10E230000C80CE70F61AF6B2012E07D13846294668
:10E240004A464346BDE8F04700F0CAB90020BDE8A1
:10E25000F08700BFB88FFF1F014B00201960704787
:10E260005C90FF1F024B0979197100F08DBF00BF50
:10E270005C90FF1F13B5002402AA1C80044B42F8D7
:10E28000041D0979197100F08DFF02B010BD00BFA7
:10E290005C90FF1F00201880014B4A88DA8070478D
:10E2A0005C90FF1F30B50C460221198021796488EB
:10E2B000084D012C297103D1BDE8304000F08ABF20
:10E2C000022C03D1BDE8304000F090BF0020188040
:10E2D00030BD00BF5C90FF1F30B50C460221198095
:10E2E00021796488084D012C297103D1BDE83040A3
:10E2F00000F088BF022C03D1BDE8304000F094BF8D
:10E300000020188030BD00BF5C90FF1F044B054A01
:10E3100019791B7A1171137203210A23FFF758BF71
:10E320005C90FF1F4C80FF1F70B500261E808B780D
:10E330000E4CC3F340014A00637261F3000203F024
:10E340000103A37205462272FFF7E0FF23685BB169
:10E35000617A01F0020101F0FF02284611B1222189
:10E36000324600E021219847002070BD5C90FF1FDD
:10E3700008B50246034B12F8080B1B6805219847A5
:10E3800008BD00BF6890FF1F38B5084D04462A1D20
:10E39000012100F0CDFF20460121802200F0E0FFA6
:10E3A0002B6820780A210022984738BD6890FF1F0B
:10E3B00037B501210DF10702044600F0B9FF9DF8C1
:10E3C0000730074D802B04D1204601212A7900F027
:10E3D000C7FF2B6820780B210022984703B030BD7F
:10E3E0006890FF1F436805215A7800F0B9BF73B5E4
:10E3F0000122002405460126002100F081FF33465A
:10E4000021468DE850002846102200F057FF214693
:10E410002246284600F074FF234621468DE850002E
:10E420002846102200F04AFF31462846022200F01A
:10E4300097FF32462846062100F092FF22462846E2
:10E44000902100F08DFF044B28781B68214622465E
:10E45000984702B070BD00BF6890FF1F42783AB97C
:10E46000C178C90141F0100101F0900100F078BFBE
:10E47000704773B50C468DF8070001F0FBF91F4E8D
:10E4800034600446002836D110211D4A9DF807004B
:10E4900000F09CFF122104461A4A9DF8070000F084
:10E4A00095FF2043C4B21421174A9DF8070000F0DD
:10E4B0008DFF2043C4B21321144A9DF8070000F0D9
:10E4C00085FF2043C4B21721114A9DF8070000F0D0
:10E4D0007DFF02AD2043C4B2162115F8010D0D4A8F
:10E4E00000F074FF2043C4B201212846032200F04B
:10E4F00037FF03233371204602B070BD6890FF1FC1
:10E50000EFE30000E5E3000089E30000B1E3000071
:10E510005DE4000071E3000037B502AC174B04F86E
:10E52000010D0022102120461A6000F051FF122137
:10E530000546204600F04CFF2843C5B21421204672
:10E5400000F046FF2843C5B21321204600F040FFEB
:10E550002843C5B21721204600F03AFF2843C5B230
:10E560001621204600F034FF284310F0FF0003D1AD
:10E570009DF8070001F08AF903B030BD6890FF1FD5
:10E5800030B585B004AC012104F8090D0DF10E027F
:10E59000204600F0CDFE204606210DF10F0200F0CE
:10E5A000C7FE9DF80E30802B16D19DF80F309B07CB
:10E5B00012D59DF8070000F0E1FD012805460BD1BA
:10E5C00072B6204600F038FB0022204629468DF81E
:10E5D0000E2000F0C5FE62B69DF80E0005B030BDFD
:10E5E00073B50E4615461C468DF80700FFF7C8FFA9
:10E5F000802807D00DF1070031462A46234600F057
:10E60000B9FA00E0002002B070BD7047062812D8A9
:10E6100080000129C0B204BF0230C0B2074AC0F373
:10E620004703122101FB03231A884FF6FF739A4216
:10E6300008BFFF207047FF20704700BF7090FF1F8A
:10E640002DE9F041334D344C344E002785F80071EC
:10E650004FF4107284F8400288462046FF2102F0F1
:10E6600011F9304639464FF48062C4F8446202F032
:10E6700009F995F80C3143F0800385F80C3195F8D1
:10E680000C21244B1206FAD4254AFF21117093F86D
:10E690000C2142F0400283F80C21A3F52C331A68B8
:10E6A000B8F1000F02D042F0004201E022F0004237
:10E6B0001A60184B320A02F0FE0283F89C20C6F35F
:10E6C000074283F8B020360E164A83F8B460C4F8C7
:10E6D0004822102283F80821012283F89420BF22C7
:10E6E00083F8802093F8002102F07F0283F8002154
:10E6F00093F8842042F0010283F8842093F8842068
:10E7000042F0100283F8842084221A770020BDE8AA
:10E71000F08100BF002007407090FF1F009AFF1F8C
:10E720005680FF1F009CFF1F0D4B93F80C2102F039
:10E73000BF0283F80C21BF2283F8802093F8842045
:10E7400002F0FE0283F8842093F8942002F0FE0287
:10E7500083F894201A7F02F07B021A77002070471A
:10E76000002007402DE9F3410B460D788C78454990
:10E7700003C902AE06E90300B3F80310B1F5007F48
:10E7800003D90021D97002211971062D19D8AF00C3
:10E79000012CF9B201D10231C9B249083A484FF00F
:10E7A000120C0CFB01FC00EB0C014FF6FF76B1F8EC
:10E7B0000080B045064604D193F80180B8F1030FFC
:10E7C00001D995205BE0012CFBD891F80F80B8F1BE
:10E7D000FF0F04BF4FF0000881F80F80B3F80380EB
:10E7E00020F80C808A73CA7BD6F84802C1F8020070
:10E7F00002F0010247EA44071743FFB2CF735A7889
:10E800004A74D6F844220C7402EBC70CB3F80380A8
:10E81000ACF80280CCF804004FF0080C02F837C0C6
:10E82000CF7BB3F8038087F0010702EBC70CCCF86D
:10E830000400ACF802804FF0480C02F837C0B3F87F
:10E8400003703844C6F8480234B9C97B12F8310065
:10E8500060F07F0002F8310058780C4A02AB03EBFD
:10E8600084042DB254F8083C12F82510012818BF72
:10E8700043F001030B43DBB202F82530002002B065
:10E88000BDE8F081F40D01007090FF1FC02007402B
:10E89000084610B51146FFF7B9FEFF281CD00F4BF4
:10E8A0001222C0F3470002FB0030D3F84432C27B8F
:10E8B00013F8324004F07F0403F8324082F0010183
:10E8C00013F8312002F07F0203F831204FF0FF33BC
:10E8D0008372C372002010BDC42010BD7090FF1F52
:10E8E00073B50D468DF80700084611461646FFF72A
:10E8F0008DFEFF2804461FD0294632460DF1070041
:10E90000FFF7C6FFC4F3470312210D4C59436318A8
:10E91000D4F848221888121AC4F848222DB2094A9D
:10E92000002002F825004FF0FF3262545A709A70AE
:10E93000DA701A715A7100E0962002B070BD00BF03
:10E940007090FF1FC02007402DE9F04180460E4621
:10E95000084611461746FFF759FE0C4CC0F3470016
:10E96000122303FB0040C57BFF2D0DD03A464046E5
:10E970003146FFF78DFF2DB2D4F8443213F835201D
:10E9800062F07B0203F83520BDE8F0817090FF1F34
:10E9900010B5084600211446FFF738FE084B122236
:10E9A000C0F3470002FB0030D3F84432C27B03EBD4
:10E9B000C2035A68136823605368636010BD00BFC8
:10E9C0007090FF1F10B508460C461146FFF71EFE5B
:10E9D000FF281AD024B2104B13F82430DBB213F006
:10E9E0000C0F12D09B0712D40C4BD3F8443213F8FF
:10E9F0003020D2090DD180F00100C0B213F83030C0
:10EA0000DB090CBF0020032010BD052010BD012034
:10EA100010BD032010BD00BFC02007407090FF1F35
:10EA200008B5FFF7F3FD074B1222C0F3470002FBC6
:10EA30000030C27BFF2A04D0D3F84432002103F80F
:10EA4000321008BD7090FF1F2DE9F04108460021EB
:10EA50001E461746FFF7DAFD244BC0F34700122588
:10EA600005FB0035EC7BFF2C3CD0B5F80080D3F8DB
:10EA700044121FFA88F24FF6FF739A4232D084F0A4
:10EA8000010311F83330C3F3C013D8B250BB4FEABF
:10EA9000C40C8EB901EB0C033046A3F80280D5F804
:10EAA00002205A6011F8343003F0400363F077031A
:10EAB00001F83430BDE8F0812B736B7301EB0C036C
:10EAC0006E81964228BF1646C5F806705E805F606C
:10EAD00011F8343003F0400363F0770301F8343069
:10EAE000BDE8F0819420BDE8F08100BF7090FF1F69
:10EAF0002DE9F04107460C46084611461546FFF73A
:10EB000085FD1A4BC0F34700122606FB0036184657
:10EB1000F17BFF2927D022B2154B84B196F811C0A2
:10EB2000012D14BF18261426BCF1010F18BF46F0A2
:10EB3000010613F822C046EA0C0603F8226013F817
:10EB400022606FF3410603F82260D0F844320022BD
:10EB500003F831203DB9384621462A462B46BDE808
:10EB6000F041FFF771BFBDE8F08100BF7090FF1F5B
:10EB7000C02007402DE9F84308460F460121904682
:10EB80009946FFF743FDFF2832D01B4AC0F34700E8
:10EB9000122404FB0024D2F84452E67B15F83630E8
:10EBA000DB0905EBC60223D139B2144B13F821104F
:10EBB00001F0020101F0FF00D1B92188C4F80680FC
:10EBC0001FFA89F363818B42A8BF0B4620736073E1
:10EBD0005380C2F804800FB9C82305E015F8363019
:10EBE00003F0400363F0770305F83630BDE8F8839F
:10EBF0009320BDE8F88300BF7090FF1FC02007403E
:10EC0000034B044883F8981001210A4600F0A8BB82
:10EC100000200740B092FF1F054B0648002283F8F2
:10EC20009420802283F80C210121FF2200F098BB60
:10EC300000200740B092FF1F38B51A4B93F800210F
:10EC400002F07F0283F8002193F80C2102F0DF022A
:10EC500083F80C2193F8802042F0200283F8802072
:10EC600093F8842002F0DF0283F8842093F8942044
:10EC700002F0DF0283F8942093F8942042F004021B
:10EC800083F8942044F620641D46013CA4B200F0B1
:10EC90009DFE002CF9D195F8943003F0FB0385F824
:10ECA000943038BD002007402DE9FF47BA4CBB4DDA
:10ECB00094F84022039995F8803095F8847095F87F
:10ECC00090608DF80420002262F317210391012146
:10ECD0008DF8062002928DF807208DF80C201F4039
:10ECE0000DEB0102FF2304F510708DF801308DF853
:10ECF000053000F01DFB95F80C31D907F6B20FD5A1
:10ED00009DF80130802B0BD195F8003103F07F0383
:10ED100085F8003195F80C3103F0DF0385F80C31EC
:10ED20007A0711D59D4B042093F8A41093F8A020E6
:10ED300083F8800004AB42EA012223F80E2D122052
:10ED400001A9029300F056FBFB0749D5934D924869
:10ED50000123BF2785F8803085F8887095F89430B6
:10ED6000002643F0020385F89430FF2185F898606F
:10ED70004FF4107285F8006101F084FD31464FF4C4
:10ED80008062D4F8440201F07DFDD4F8443203F5EA
:10ED90000073C4F84832824BFF221A7095F8943001
:10EDA00003F0FD0385F8943095F80C3143F04003EF
:10EDB00085F80C319F2385F88C7085F8843095F8A0
:10EDC000943003F0DF0385F89430102001A900F09F
:10EDD00011FB95F8943003F0DF0385F8943061E17E
:10EDE0003D0740F1F4806D4B082283F88020320902
:10EDF000C6F3C001062A8DF805208DF8071007D844
:10EE0000C6F3800303EB820319B10233DBB200E0E7
:10EE1000FF23D4F84452D90068185A084FF0120C56
:10EE20000CFB0244426802924088ADF80D00E07B82
:10EE300080F00100E07383F0010615F83330C3F36E
:10EE4000801383F001039B0105F836309DF80730ED
:10EE50009DF80590012B05EBC60843D1DFF840A1D2
:10EE6000B9F1000F14D19AF80090B9F1000F0FD149
:10EE7000FF2349464A4601A88AF80030FFF708FDFB
:10EE800005F8369001A849464A464B46FFF7DCFD97
:10EE90009AF80030012B04D09DF80530002B00F0CB
:10EEA0008A80BDF80DC0A38960892288D4F8061035
:10EEB00063449BB29842A38106D85FFA8CFC6245FA
:10EEC0000CD1A47B012C09D11944C31A9342D8BF99
:10EED0009AB2A8F80220C8F8041053E00291ADF8E5
:10EEE0000D3068E0B9F1000F1DD16B5CC3F38303F3
:10EEF0000D2B2B4B06D101218DF806101278D2096B
:10EF00001A7010E01A78012A0DD1FF21197001A89A
:10EF10004946FFF7BDFC05F8369001A849464A4628
:10EF20004B46FFF791FD62894FF6FF739A4242D03C
:10EF3000BDF80D00A1892388014489B29842A181BE
:10EF400001D18A4209D86AB3B2FBF3F003FB102067
:10EF500080B238BBA07B012824D1521A9A42D8BF74
:10EF600093B243B9D4F80220C8F8042088F80230DC
:10EF700088F8033006E0D4F80620A8F802301144DF
:10EF8000C8F8041015F8363003F0400363F0770337
:10EF900005F8363014E000BF7090FF1F00200740D6
:10EFA0005680FF1FD4F8063002934FF0FF33ADF8C0
:10EFB0000D10A372E3729DF8050001A900F01AFA82
:10EFC0003A4B93F8942002F0DF0283F89420B807BC
:10EFD00017D5364C022384F8803094F8883094F8A2
:10EFE0008C201620134001A98DF80C3000F002FA95
:10EFF000BF2384F8883094F8943003F0DF0384F85A
:10F000009430F9061CD5294C202384F88030102335
:10F0100084F88030142001A900F0ECF994F80C3148
:10F0200043F0200384F80C3194F8003143F080035E
:10F0300084F8003194F8843043F0200384F884305D
:10F04000BA060DD5194C202384F88030132001A96D
:10F0500000F0D0F994F8843003F0DF0384F88430B2
:10F060003B061FD5FF2301A810210DF102028DF8E8
:10F07000053000F05DF99DF80230012B04D100222B
:10F080008DF805208DF80730084C802384F88030F7
:10F09000172001A900F0AEF994F8943003F0DF03D3
:10F0A00084F8943004B0BDE8F08700BF002007402A
:10F0B0000B4611461A4601F0E5BB00BF30B50329E7
:10F0C000039D049C1CD123B9164A2A600422228085
:10F0D00026E040F209418B4205D1022A4FF000039D
:10F0E00003D9012201E001231A460F490C2000FB3D
:10F0F0000313D9681B6951F8221029609B5C0EE04C
:10F10000072901D9CD2030BD074B03EB8102126ADC
:10F110002A60002AF6D003EB4101B1F84030238089
:10F12000002030BD5780FF1FFC0D0100012904D8CD
:10F13000034B5B5C137000207047CD20704700BF0D
:10F14000BC92FF1F01299DBF024B00205A54CD20C5
:10F15000704700BFBC92FF1F01298CBF0020012017
:10F160007047054B1A788A4204D05878431A58429F
:10F170005841704701207047BC92FF1F0020704724
:10F18000004870474C0E0100012906D8044BC1EB22
:10F19000C1011944116000207047CD20704700BFA5
:10F1A0005B80FF1F012910B50DD8094BC1EBC101D0
:10F1B000194408231068C45CC81801330F2B00F8E9
:10F1C000084CF7D101E0CD2010BD002010BD00BFDC
:10F1D0005B80FF1F012905D8034B03EB4101116040
:10F1E00000207047CD207047BE92FF1F012905D82F
:10F1F000034B03EB4101116000207047CD207047A5
:10F20000C292FF1F01290AD80648136800EB41018A
:10F210001B788B7013685B78CB7000207047CD2013
:10F22000704700BFBC92FF1F01290AD80648136827
:10F2300000EB41011B788B7113685B78CB71002068
:10F240007047CD20704700BFBC92FF1F084B5A7813
:10F250001A700023074AFF2199540133072BF9D173
:10F260000023054A052199540133072BF9D1704732
:10F27000C692FF1FC892FF1FCF92FF1F00BF7047AB
:10F28000013AD2B2062A38B505461C4609D8064BC3
:10F290005A70FFF7DBFF28462146BDE83840FFF7EC
:10F2A000CFB9992038BD00BFC692FF1F024B002284
:10F2B0005A70FFF739BA00BFC692FF1F37B50F4C1F
:10F2C000257805B9B9B98DF802308DF800109DF890
:10F2D0001830ADF8032000789DF81C208DF801301F
:10F2E0006946FFF73FFA9DF800302BB120B923782B
:10F2F000013B237000E0952003B030BDC692FF1F94
:10F3000038B50A4B0C461D7859788D421D4600D100
:10F310004CB900782146FFF7E3FA2CB120B92B78DD
:10F3200001332B7038BD962038BD00BFC692FF1F39
:10F330004B1E062B03D8094B19444B7808E0CB062B
:10F3400009D501F00F01062905D8044B19444B7A61
:10F350001370002070478220704700BFC692FF1FC5
:10F360004B1E062B2DE9F0418046154603D8164B5F
:10F3700019444A7021E0CB0622D501F00F04062C77
:10F380001ED8012A4FEAD1160F4F04D1214632462A
:10F39000FFF7DAFA0FE072B93B195B7A012B0AD159
:10F3A00021463246FFF7A4FB2CB94046214686F0A1
:10F3B0000102FFF79DFB3C4465720020BDE8F0812F
:10F3C0008220BDE8F08100BFC692FF1F0020704779
:10F3D000062903D9A1F11003072B07D8044B53F8D2
:10F3E0002130002B14BF0020C4207047C420704778
:10F3F000740E0100102838B504460D4601D1FFF700
:10F4000025FF044B53F824300BB1284698470020C1
:10F4100038BD00BF740E01001FB504A9144601F8E1
:10F42000090D02221A8008460DF10F020521FFF78F
:10F430007FFF034B9DF80F201A80236004B010BD9E
:10F44000D892FF1F1FB504A9144601F8090D012227
:10F450001A8008460DF10F020421FFF769FF044BE3
:10F460009DF80F201A800020236004B010BD00BF5B
:10F47000D892FF1F7FB500241C8049888DF80700B3
:10F48000ADF80E10FFF768FE00B3BDF80E20114E68
:10F49000131B5A425A410DF107000121FFF760FF8B
:10F4A0009DF80E200DF107000421FFF759FF736846
:10F4B0000DF10E02054601219DF80700984773687B
:10F4C0009DF8070002212246984700E004252846BF
:10F4D00004B070BDD892FF1F37B502AA002402F80D
:10F4E000010D0D461C80104601210422FFF738FF54
:10F4F0006A88024B20461A7203B030BDD892FF1FB3
:10F5000037B54C888D888DE80C00210AE2B22B4675
:10F51000FFF7D4FD03B030BD2DE9F04186B00F46B2
:10F520001E4600238DF80F000593904603230DF12E
:10F530000F00012104AA8DF81030FFF7F9FE3D7885
:10F54000274C15F0030525D106210DF111020DF10F
:10F550000F00FFF7EDFE9DF811309DF80F0003F04E
:10F560000303238005AB00930DF1120301930221E5
:10F570002B462A46FFF7A2FD059BDB7913F0400FCF
:10F58000238814BF43F0010323F0010323800223E7
:10F5900033801FE0012D09D19DF81020BB88012A7E
:10F5A00002D113F0FF0F14D10023EFE7022D11D188
:10F5B000397941F010010DF10F00C9B20DF11202BD
:10F5C000FFF7B6FE9DF8123003F00103238035806B
:10F5D00000E0CD20C8F8004006B0BDE8F08100BFD3
:10F5E000D892FF1F7FB500221A800B784E788DF8D5
:10F5F000070013F003030D46C6F3400632D1B6B13F
:10F600004B88013B9BB2012B50D80DF1070006211E
:10F610000DF10F02FFF78CFE0446002847D1AA78AF
:10F620009DF80F3006FA02F21A43D2B211E04E886A
:10F63000012E3BD10DF1070006210DF10F02FFF75E
:10F6400077FE044698BBAA789DF80F30964023EACF
:10F6500006020DF1070006218DF80F20FFF780FE4E
:10F66000044624E0022B21D109798DF80F100DF109
:10F67000070041F010013246FFF772FE6B78002E52
:10F680000CBF08210721012B044607D19DF80F105C
:10F6900001F00F00C909FFF7C3F90821054B9DF8D8
:10F6A00007005B680DF10F02984700E0CD2420466B
:10F6B00004B070BDD892FF1F10B500241C800B78D9
:10F6C00003F00303012B0A4605D109799278FFF76D
:10F6D00039FD204610BD042010BD38B50C7804F06B
:10F6E0000304012C154607D11C80044C09792246DD
:10F6F000FFF71CFD2C6038BD042038BDD892FF1FD9
:10F7000013B5CD298DF8070006D10DF10700902122
:10F710000122FFF725FE18E00D481C88018A1268B7
:10F720008C4288BF198004461B889DF80700002181
:10F73000FEF756FF94F90A30002B06DA00210DF18E
:10F7400007000A460B46FFF77FF902B010BD00BF65
:10F75000D892FF1F73B5054600266A4601218DF831
:10F7600000600196FFF7E4FDAA783F4C012A46D1DC
:10F7700068680368C4F80A304368A07AC4F80E3099
:10F7800004F10A0110F0600F238A13D1E37A37489D
:10F7900050F82340002C5ED09DF80020022A5AD851
:10F7A00003EB43031844024492F83430012B52D146
:10F7B000287818E0202BADF802301AD873B1020671
:10F7C0000CD40A68C4F812204A68C4F816202846E7
:10F7D000314604F11A02FFF737F943E0E46B002CDD
:10F7E00039D02878224901AA0DF10203A047014629
:10F7F00032E002A82B7800F8073D902113E09DF835
:10F800000030042B12D12B78217A02AD05F8063D89
:10F810002846FFF7F5F901210A462846FFF7A0FD23
:10F82000227A28460321FFF79BFD1BE094F90A305A
:10F83000002B17DBEB78ABB9E66B66B1B5F8093096
:10F8400028780833ADF8023004F1120101AA0DF155
:10F850000203B047CBE7CD21287801AA0DF10203BE
:10F86000FFF74EFF02B070BDD892FF1FD40E01000B
:10F87000E292FF1F034B5960DA630021024AFFF74F
:10F88000A5BD00BFD892FF1F55F7000007B502AB1A
:10F89000054A03F8010D002118465160D163FFF7B6
:10F8A00097FD03B05DF804FBD892FF1F002070475E
:10F8B000354B41F24802995821F00F0141F0020105
:10F8C000995041F20402995841F48021995041F233
:10F8D0003402995841F48021995003F52C3360216A
:10F8E00093F8942042F0020283F89420C02283F817
:10F8F0000021FF221A7483F8802083F8882083F87F
:10F900008420002283F88C2083F80C111F491A757B
:10F91000080A00F0FE0083F8982083F8C02083F8DE
:10F92000C42083F8C82083F8CC2083F8D02083F843
:10F93000D42083F8D82083F8DC2083F8E02083F8F3
:10F94000E42083F8E82083F8EC2083F8F02083F8A3
:10F95000F42083F8F82083F8FC2083F89C00C1F39E
:10F960000740090E83F8B00083F8B41083F8AC2088
:10F970001A7783F8082193F8942002F0D40242F019
:10F98000010283F89420704700700440009AFF1F22
:10F99000024B4FF400125A60704700BF00E100E0D4
:10F9A000034B4FF40012C3F884215A60704700BF24
:10F9B00000E100E010B5FEF78DF9044618B9FFF735
:10F9C000EFFF204610BD1B2010BD00BF034B4AF2C5
:10F9D00002629A814BF280429A8170470020054072
:10F9E00081F0004102E000BF83F0004330B54FEAF0
:10F9F00041044FEA430594EA050F08BF90EA020F5D
:10FA00001FBF54EA000C55EA020C7FEA645C7FEAEF
:10FA1000655C00F0E2804FEA5454D4EB5555B8BF12
:10FA20006D420CDD2C4480EA020281EA030382EA83
:10FA3000000083EA010180EA020281EA0303362D15
:10FA400088BF30BD11F0004F4FEA01314FF4801CE8
:10FA50004CEA113102D0404261EB410113F0004FFA
:10FA60004FEA03334CEA133302D0524263EB4303B1
:10FA700094EA050F00F0A780A4F10104D5F1200E4F
:10FA80000DDB02FA0EFC22FA05F2801841F10001AA
:10FA900003FA0EF2801843FA05F359410EE0A5F17E
:10FAA00020050EF1200E012A03FA0EFC28BF4CF0AF
:10FAB000020C43FA05F3C01851EBE37101F0004565
:10FAC00007D54FF0000EDCF1000C7EEB00006EEB72
:10FAD0000101B1F5801F1BD3B1F5001F0CD34908FC
:10FAE0005FEA30004FEA3C0C04F101044FEA445253
:10FAF00012F5800F80F09A80BCF1004F08BF5FEADA
:10FB0000500C50F1000041EB045141EA050130BDB9
:10FB10005FEA4C0C404141EB010111F4801FA4F15C
:10FB20000104E9D191F0000F04BF01460020B1FAB1
:10FB300081F308BF2033A3F10B03B3F120020CDAE9
:10FB40000C3208DD02F1140CC2F10C0201FA0CF0C7
:10FB500021FA02F10CE002F11402D8BFC2F1200C2C
:10FB600001FA02F120FA0CFCDCBF41EA0C019040E2
:10FB7000E41AA2BF01EB0451294330BD6FEA04042B
:10FB80001F3C1CDA0C340EDC04F11404C4F1200216
:10FB900020FA04F001FA02F340EA030021FA04F328
:10FBA00045EA030130BDC4F10C04C4F1200220FA7F
:10FBB00002F001FA04F340EA0300294630BD21FABD
:10FBC00004F0294630BD94F0000F83F4801306BF83
:10FBD00081F480110134013D4EE77FEA645C18BF77
:10FBE0007FEA655C29D094EA050F08BF90EA020F0E
:10FBF00005D054EA000C04BF1946104630BD91EA06
:10FC0000030F1EBF0021002030BD5FEA545C05D108
:10FC10004000494128BF41F0004130BD14F5800447
:10FC20003CBF01F5801130BD01F0004545F0FE41BB
:10FC300041F470014FF0000030BD7FEA645C1ABFF0
:10FC4000194610467FEA655C1CBF0B46024650EA27
:10FC5000013406BF52EA033591EA030F41F4002153
:10FC600030BD00BF90F0000F04BF0021704730B5D9
:10FC70004FF4806404F132044FF000054FF00001AE
:10FC800050E700BF90F0000F04BF0021704730B56F
:10FC90004FF4806404F1320410F0004548BF404244
:10FCA0004FF000013EE700BF42004FEAE2014FEA99
:10FCB00031014FEA02701FBF12F07F4393F07F4F74
:10FCC00081F06051704792F0000F14BF93F07F4FA6
:10FCD000704730B54FF4607401F0004521F00041E9
:10FCE00020E700BF50EA010208BF704730B54FF06F
:10FCF00000050AE050EA010208BF704730B511F074
:10FD0000004502D5404261EB41014FF4806404F1AB
:10FD100032045FEA915C3FF4DCAE4FF003025FEA2D
:10FD2000DC0C18BF03325FEADC0C18BF033202EBB5
:10FD3000DC02C2F1200300FA03FC20FA02F001FA0F
:10FD400003FE40EA0E0021FA02F11444C1E600BFAE
:10FD500070B54FF0FF0C4CF4E06C1CEA11541DBF61
:10FD60001CEA135594EA0C0F95EA0C0F00F0DEF82C
:10FD70002C4481EA030621EA4C5123EA4C5350EA11
:10FD8000013518BF52EA033541F4801143F4801362
:10FD900038D0A0FB02CE4FF00005E1FB02E506F0F3
:10FDA0000042E0FB03E54FF00006E1FB03569CF048
:10FDB000000F18BF4EF0010EA4F1FF04B6F5007F4E
:10FDC00064F5407404D25FEA4E0E6D4146EB0606C0
:10FDD00042EAC62141EA55514FEAC52040EA5E5049
:10FDE0004FEACE2EB4F1FD0C88BFBCF5E06F1ED8F3
:10FDF000BEF1004F08BF5FEA500E50F1000041EB2A
:10FE0000045170BD06F0004646EA010140EA0200D6
:10FE100081EA0301B4EB5C04C2BFD4EB0C0541EAF8
:10FE2000045170BD41F480114FF0000E013C00F30D
:10FE3000AB8014F1360FDEBF002001F0004170BD31
:10FE4000C4F10004203C35DA0C341BDC04F114044A
:10FE5000C4F1200500FA05F320FA04F001FA05F2D6
:10FE600040EA020001F0004221F0004110EBD370A3
:10FE700021FA04F642EB06015EEA430E08BF20EACF
:10FE8000D37070BDC4F10C04C4F1200500FA04F372
:10FE900020FA05F001FA04F240EA020001F0004104
:10FEA00010EBD37041F100015EEA430E08BF20EA77
:10FEB000D37070BDC4F1200500FA05F24EEA020EBF
:10FEC00020FA04F301FA05F243EA020321FA04F0EE
:10FED00001F0004121FA04F220EA020000EBD370A5
:10FEE0005EEA430E08BF20EAD37070BD94F0000FA5
:10FEF0000FD101F00046400041EB010111F4801FD9
:10FF000008BF013CF7D041EA060195F0000F18BF89
:10FF1000704703F00046520043EB030313F4801FC5
:10FF200008BF013DF7D043EA0603704794EA0C0F7F
:10FF30000CEA135518BF95EA0C0F0CD050EA410695
:10FF400018BF52EA4306D1D181EA030101F0004112
:10FF50004FF0000070BD50EA410606BF104619463A
:10FF600052EA430619D094EA0C0F02D150EA013646
:10FF700013D195EA0C0F05D152EA03361CBF104687
:10FF800019460AD181EA030101F0004141F0FE4126
:10FF900041F470014FF0000070BD41F0FE4141F4AA
:10FFA000780170BD70B54FF0FF0C4CF4E06C1CEAAA
:10FFB00011541DBF1CEA135594EA0C0F95EA0C0F5F
:10FFC00000F0A7F8A4EB050481EA030E52EA03351A
:10FFD0004FEA013100F088804FEA03334FF080553B
:10FFE00045EA131343EA12634FEA022245EA111568
:10FFF00045EA10654FEA00260EF000419D4208BF19
:020000021000EC
:10000000964244F1FD0404F5407402D25B084FEAC5
:100010003202B61A65EB03055B084FEA32024FF471
:1000200080104FF4002CB6EB020E75EB030E22BFCE
:10003000B61A754640EA0C005B084FEA3202B6EB8E
:10004000020E75EB030E22BFB61A754640EA5C003D
:100050005B084FEA3202B6EB020E75EB030E22BFCD
:10006000B61A754640EA9C005B084FEA3202B6EBCE
:10007000020E75EB030E22BFB61A754640EADC008D
:1000800055EA060E18D04FEA051545EA16754FEAEF
:1000900006164FEAC30343EA52734FEAC2025FEA0D
:1000A0001C1CC0D111F4801F0BD141EA00014FF09C
:1000B00000004FF0004CB6E711F4801F04BF01436D
:1000C0000020B4F1FD0C88BFBCF5E06F3FF6AFAE89
:1000D000B5EB030C04BFB6EB020C5FEA500C50F119
:1000E000000041EB045170BD0EF0004E4EEA11319C
:1000F00014EB5C04C2BFD4EB0C0541EA045170BDA3
:1001000041F480114FF0000E013C90E645EA060EE6
:100110008DE60CEA135594EA0C0F08BF95EA0C0F14
:100120003FF43BAF94EA0C0F0AD150EA01347FF45C
:1001300034AF95EA0C0F7FF425AF104619462CE733
:1001400095EA0C0F06D152EA03353FF4FDAE104696
:10015000194622E750EA410618BF52EA43067FF4E7
:10016000C5AE50EA41047FF40DAF52EA43057FF477
:10017000EBAE12E74FF0FF3C06E000BF4FF0010C82
:1001800002E000BF4FF0010C4DF804CD4FEA410CE6
:100190007FEA6C5C4FEA430C18BF7FEA6C5C1BD0B3
:1001A00001B050EA410C0CBF52EA430C91EA030F34
:1001B00002BF90EA020F0020704710F1000F91EA91
:1001C000030F58BF994208BF90422CBFD8176FEA5F
:1001D000E37040F0010070474FEA410C7FEA6C5C2D
:1001E00002D150EA013C07D14FEA430C7FEA6C5C34
:1001F000D6D152EA033CD3D05DF8040B704700BF60
:100200008446104662468C461946634600E000BFAD
:1002100001B5FFF7B7FF002848BF10F1000F01BD7F
:100220004DF808EDFFF7F4FF0CBF012000205DF84A
:1002300008FB00BF4DF808EDFFF7EAFF34BF0120CF
:1002400000205DF808FB00BF4DF808EDFFF7E0FF68
:1002500094BF012000205DF808FB00BF4DF808EDB9
:10026000FFF7CEFF94BF012000205DF808FB00BF20
:100270004DF808EDFFF7C4FF34BF012000205DF802
:1002800008FB00BF4FEA410212F5001215D211D54A
:100290006FF47873B3EB625212D94FEAC12343F083
:1002A000004343EA505311F0004F23FA02F018BF05
:1002B000404270474FF00000704750EA013005D1CE
:1002C00011F0004008BF6FF0004070474FF0000091
:1002D000704700BF80F0004002E000BF81F00041A5
:1002E00042001FBF5FEA410392EA030F7FEA226CDC
:1002F0007FEA236C6AD04FEA1262D2EB1363C1BF6C
:10030000D218414048404140B8BF5B42192B88BFDA
:10031000704710F0004F40F4000020F07F4018BFFD
:10032000404211F0004F41F4000121F07F4118BF1D
:10033000494292EA030F3FD0A2F1010241FA03FCC5
:1003400010EB0C00C3F1200301FA03F100F00043AD
:1003500002D5494260EB4000B0F5000F13D3B0F175
:10036000807F06D340084FEA310102F10102FE2AE4
:1003700051D2B1F1004F40EBC25008BF20F0010054
:1003800040EA03007047490040EB000010F4000F02
:10039000A2F10102EDD1B0FA80FCACF1080CB2EB95
:1003A0000C0200FA0CF0AABF00EBC25052421843F4
:1003B000BCBFD0401843704792F0000F81F4000199
:1003C00006BF80F400000132013BB5E74FEA41036C
:1003D0007FEA226C18BF7FEA236C21D092EA030FD8
:1003E00004D092F0000F08BF0846704790EA010F52
:1003F0001CBF0020704712F07F4F04D1400028BF7F
:1004000040F00040704712F100723CBF00F5000060
:10041000704700F0004343F0FE4040F40000704796
:100420007FEA226216BF08467FEA23630146420242
:1004300006BF5FEA412390EA010F40F48000704755
:100440004FF0000304E000BF10F0004348BF4042FB
:100450005FEA000C08BF704743F0964301464FF037
:1004600000001CE050EA010208BF70474FF0000393
:100470000AE000BF50EA010208BF704711F00043D4
:1004800002D5404261EB41015FEA010C02BF8446A4
:100490000146002043F0B64308BFA3F18053A3F503
:1004A0000003BCFA8CF2083AA3EBC25310DB01FA4A
:1004B00002FC634400FA02FCC2F12002BCF1004FCE
:1004C00020FA02F243EB020008BF20F0010070475F
:1004D00002F1200201FA02FCC2F1200250EA4C00B3
:1004E00021FA02F243EB020008BF20EADC707047F9
:1004F0004FF0FF0C1CEAD0521EBF1CEAD15392EA07
:100500000C0F93EA0C0F6FD01A4480EA010C4002E2
:1005100018BF5FEA41211ED04FF0006343EA50103C
:1005200043EA5111A0FB01310CF00040B1F5000F7E
:100530003EBF490041EAD3715B0040EA010062F12D
:100540007F02FD2A1DD8B3F1004F40EBC25008BF17
:1005500020F00100704790F0000F0CF0004C08BF35
:1005600049024CEA502040EA51207F3AC2BFD2F102
:10057000FF0340EAC250704740F400004FF0000310
:10058000013A5DDC12F1190FDCBF00F0004070474A
:10059000C2F10002410021FA02F1C2F1200200FA88
:1005A00002FC5FEA310040F1000053EA4C0308BF4F
:1005B00020EADC70704792F0000F00F0004C02BFA0
:1005C000400010F4000F013AF9D040EA0C0093F01B
:1005D000000F01F0004C02BF490011F4000F013B75
:1005E000F9D041EA0C018FE70CEAD15392EA0C0FE3
:1005F00018BF93EA0C0F0AD030F0004C18BF31F04E
:10060000004CD8D180EA010000F00040704790F023
:10061000000F17BF90F0004F084691F0000F91F0C7
:10062000004F14D092EA0C0F01D142020FD193EA8D
:100630000C0F03D14B0218BF084608D180EA010015
:1006400000F0004040F0FE4040F40000704740F0F1
:10065000FE4040F4400070474FF0FF0C1CEAD052BF
:100660001EBF1CEAD15392EA0C0F93EA0C0F69D01B
:10067000A2EB030280EA010C49024FEA402037D086
:100680004FF0805343EA111143EA10130CF000407D
:100690008B4238BF5B0042F17D024FF4000C8B426D
:1006A00024BF5B1A40EA0C00B3EB510F24BFA3EB4D
:1006B000510340EA5C00B3EB910F24BFA3EB91031D
:1006C00040EA9C00B3EBD10F24BFA3EBD10340EA77
:1006D000DC001B0118BF5FEA1C1CE0D1FD2A3FF6BD
:1006E00050AF8B4240EBC25008BF20F00100704772
:1006F0000CF0004C4CEA50207F32C2BFD2F1FF0315
:1007000040EAC250704740F400004FF00003013A45
:1007100037E792F0000F00F0004C02BF400010F4E9
:10072000000F013AF9D040EA0C0093F0000F01F0FD
:10073000004C02BF490011F4000F013BF9D041EA1F
:100740000C0195E70CEAD15392EA0C0F08D1420252
:100750007FF47DAF93EA0C0F7FF470AF084676E725
:1007600093EA0C0F04D14B023FF44CAF08466EE7FE
:1007700030F0004C18BF31F0004CCAD130F00042CC
:100780007FF45CAF31F000437FF43CAF5FE700BF24
:10079000FDF737F9002100F004B80C4B5B584350CB
:1007A00004310B480B4B42189A42FFF4F6AF0A4A49
:1007B00000F003B8002313600432084B9A42FFF4A0
:1007C000F9AF00F00DF8804770470000680F010096
:1007D0000880FF1F6885FF1F0086FF1F009EFF1F08
:1007E000254C08B5F7F741FEF7F7A4FEF7F7EEFF43
:1007F000F8F702F8F7F706FFF8F7D0F9FCF7C0FAB8
:10080000FCF78CF8F8F73BFBF8F784F82078F7F75B
:1008100009FFE078F7F776FFF8F724F928B1F8F741
:1008200021F96070F8F71EF9A060F8F793F9607984
:100830002189228AFCF7CCF8FCF79EFFFCF744FBE9
:100840000E4B4FF400725A60FAF7A0FEFBF754FB10
:100850000B4B04225A60FAF7B1FFFBF78BFBFBF757
:100860004CFBF8F731F9F8F765F90028F3D0FCF7FD
:1008700083FFFAF78BFEEEE70C80FF1F80F00F403E
:1008800000F00F40F0B4840743D0541E002A3ED03D
:10089000CDB2034603E0621E002C38D0144603F8A4
:1008A000015B9A07F7D1032C2AD9CDB245EA052579
:1008B0000F2C45EA054515D9A4F110073F0903F1AE
:1008C000100606EB07161A46156055609560D56050
:1008D0001032B242F8D104F00F040137032C03EBBD
:1008E00007130DD91E462246043A032A46F8045B34
:1008F000FAD8221F22F003020432134404F0030446
:100900002CB1C9B21C4403F8011BA342FBD1F0BCBB
:10091000704714460346C6E7C1F30A5CF8B5ACF26B
:10092000FF33132B06460F4610DC002B39DBDFF8B4
:1009300088C04CFA03F303EA010C5CEA000C1AD1FC
:1009400007F000416046C2E90067F8BD332B1CDCAC
:100950004FF0FF33ACF2134C23FA0CFC1CEA0003FB
:1009600019D020EA0C060F46C2E900670B46324652
:10097000FFF73AF8F8BD21EA03070026C2E900674D
:100980003B463246FFF730F8F8BD07F00041002043
:10099000C2E90067F8BD07F000411846C2E90067E8
:1009A000F8BD07F00041002004460D4630463946A8
:1009B000C2E90045F8BD00BFFFFF0F00024B13B1B5
:1009C000024800F005B8704700000000DD09010092
:1009D000014600200246034600F018B838B5094D1C
:1009E000094C641BA41018BF05EB840505D0013C1D
:1009F00055F8043D9847002CF9D1BDE8384000F087
:100A0000A7BA00BF640F0100680F0100F0B5274CC2
:100A10002668D6F8484185B00746002C41D0656865
:100A20001F2D1EDD224818B94FF0FF3005B0F0BD74
:100A30004FF4C870039102920193AFF300800399C1
:100A4000029A019B04460028EED0D6F84851256052
:100A5000002060600546C6F84841C4F88801C4F823
:100A60008C013FB9AB1C00200135656044F82310B0
:100A700005B0F0BD04EB85004FF0010CC0F88820F4
:100A8000D4F888610CFA05F21643022FC4F8886185
:100A9000C0F80831E6D1D4F88C311A43C4F88C215F
:100AA000E0E706F5A674C6F84841B8E7400F010034
:100AB00000000000000000002DE9F84FC1F30A57C4
:100AC000A7F2FF36132E02460B4604460D46894612
:100AD0008A46804622DC002E54DB3D4F374107EA30
:100AE000010C5CEA000C1ED037A3D3E90023FEF70B
:100AF0007DFF00220023FFF7BBFB58B1002D05DD71
:100B00004FF4801A4AFA06F606EB050A2AEA0709A4
:100B10004FF0000840464946BDE8F88F332E06DD09
:100B2000B6F5806F43D010461946BDE8F88FA7F29E
:100B3000134C4FF0FF3B2BFA0CFB1BEA000FF2D0DB
:100B400021A3D3E90023FEF751FF00220023FFF782
:100B50008FFB0028DED0002D0DDD142E09D0C7F547
:100B6000866703374FF0010808FA07F818EB040806
:100B700001D305F1010A28EA0B08D146404649464F
:100B8000BDE8F88F10A3D3E90023FEF72FFF002262
:100B90000023FFF76DFB0028BCD0002D0DDB55EACC
:100BA000040808D0DFF82C904FF00008B2E7FEF7F9
:100BB0001DFFBDE8F88FC146ACE74FF000084FF0CD
:100BC0000049A7E7AFF300809C7500883CE4377EBE
:100BD000FFFF0F000000F03F2DE9F84FC1F30A5767
:100BE000A7F2FF36132E02460B4604460D468946F1
:100BF0008A4680461CDC002E40DB3D4F374107EA29
:100C0000010C5CEA000C18D037A3D3E90023FEF7EF
:100C1000EDFE00220023FFF72BFB28B1002D42DB65
:100C20002AEA07094FF0000840464946BDE8F88F18
:100C3000332E06DDB6F5806F31D010461946BDE87B
:100C4000F88FA7F2134C4FF0FF3B2BFA0CFB1BEA7B
:100C5000000FF2D024A3D3E90023FEF7C7FE002241
:100C60000023FFF705FB0028DED0002D22DB28EA59
:100C70000B08D14640464946BDE8F88F1AA3D3E990
:100C80000023FEF7B3FE00220023FFF7F1FA00284D
:100C9000CAD0002D1CDB4FF00008C146C4E7FEF7A8
:100CA000A5FEBDE8F88F4FF4801A4AFA06F606EB67
:100CB000050AB5E7142E14D0C7F58667012303375C
:100CC00003FA07F717EB040828BF05EB030ACEE782
:100CD00025F00042074B224318BF99464FF0000809
:100CE000A2E705F1010AC2E79C7500883CE4377E63
:100CF000FFFF0F000000F0BF80250000403800001B
:100D0000004B0000807000000096000000E1000031
:100D1000002C010000C201000084030090D00300F9
:100D200020A1070040420F0050C3000088130000BC
:100D3000018008080000000000000000C80000005A
:100D40000100C8000080000000000000000000005A
:100D50000000000000000000000000000000000093
:100D60000000000000000000010002000400080074
:100D7000100020000101010001000000000000003F
:100D80000000000000000100000000000000000062
:100D90000000000001010100000000000000000050
:100DA000000100000000000001010100010100013C
:100DB0000100000000000000000000000000000032
:100DC0000000000000000000000000000000000023
:100DD0000000000000000000000000000000010111
:100DE00001000001000100010000000000000000FF
:100DF0000000000008000000040000005780FF1FF2
:100E00000400000009040000600E0100700E0100E3
:100E100000000000000000000000000000000000D2
:100E20002E81FF1FEB80FF1F00000000000000006C
:100E300000000000000000000000000000001200A0
:100E40004300000000000000000000000301020158
:100E50001000020200100003030110000001000056
:100E60005780FF1FB180FF1F8B80FF1F6980FF1F0E
:100E7000043A262255F7000059E00000EDE000009A
:100E80005DDE00007DF200007DF200007DF20000DA
:100E90007DF200007DF200007DF200007DF2000096
:100EA0007DF200007DF200007DF200007DF2000086
:100EB0007DF20000EFE3000089E30000E5E30000BD
:100EC000B1E3000089E300007DF2000071E300005F
:100ED0005DE4000019F50000E5F5000000000000E9
:100EE000E5F5000000000000D9F4000001F5000065
:100EF0000000000045F4000075F40000DBF600007F
:100F0000B9F6000019F40000010100010100000021
:100F100000010100000000000101010101000000CA
:100F200001010001010001000001000001000000BA
:100F300033323132563130350000000043000000BA
:100F40004081FF1FF8B500BFF8BC08BC9E46704743
:0C0F5000F8B500BFF8BC08BC9E46704716
:080F5C00BD090100358400000D
:040F640011840000F4
:100F6800300F01000001020000080000010000002D
:100F78000200000000000000000000000000000067
:100F88000000000000000000000000000000000059
:100F98000000000000000000000000000000000049
:100FA80000000000A1200000000002000000FF0473
:100FB80003090400C201000000080000000000004E
:100FC8000022034200410044002000530054005214
:100FD8000049004E004700200049004E00440045EB
:100FE8000058002603530074006500700070006507
:100FF80000720020004D006F0074006F0072002026
:101008000044006500760020003A0354005200496D
:10101800004E0041004D004900430020004D006F84
:1010280000740069006F006E00200043006F006EBE
:1010380000740072006F006C002000200020002067
:1010480000200009024300020100C0320904000028
:101058000102020000052400100105240101010419
:1010680024020605240600010705830310000A0967
:10107800040100020A0000000705810210000007B1
:1010880005020210000012010002020000103C2AB2
:101098000001020001020001000000002C84FF1F73
:1010A8009484FF1FFC84FF1F000000000000000064
:1010B8000000000000000000000000000000000028
:1010C8000000000000000000000000003C0F0100CC
:1010D8000000000000000000000000000000000008
:1010E80000000000000000000000000000000000F8
:1010F80000000000000000000000000000000000E8
:1011080000000000000000000000000000000000D7
:1011180000000000000000000000000000000000C7
:1011280000000000000000000000000000000000B7
:1011380000000000000000000000000000000000A7
:1011480001000000000000000E33CDAB34126DE644
:10115800ECDE05000B0000000000000000000000AD
:101168000000000000000000000000000000000077
:101178000000000000000000000000000000000067
:101188000000000000000000000000000000000057
:101198000000000000000000000000000000000047
:1014C800680F01000880FF1F600500000000000091
:0814D80000000000000000000C
:020000020000FC
:020000041FFFDC
:04800000000000007C
:040000031000079151
:00000001FF
